:020000040000FA
:1000000002EF00F00F013F0E926E000E936E000E95
:10001000946E030E956E0F0E966E000E386F000EE6
:10002000396F000E3A6F000E3B6F000E3C6F806A16
:10003000816A826A836A846A896A8A6A8B6A8C6A3C
:100040008D6A00018B8C8B82006A016A026A036AE6
:10005000046A056A066A076A086A096A0A6A0B6A14
:100060000C6A0D6A0E6A0F6A106A116A126A136AC4
:10007000146A156A166A176A186A196A1A6A1B6A74
:100080001C6A1D6A1E6A1F6A206A216A226A236A24
:10009000256A266A276A296A246A286A2A6A2B6AD4
:1000A0002C6A2D6A2E6A2F6A306A316A326A336A84
:1000B000346A356A366A376A386A396A3A6A3C6A33
:1000C0003B6A3D6A3E6A3F6A406A416A426A436AE5
:1000D000446A456A466A476A486A496A4A6A4B6A94
:1000E0004C6A4D6A4E6A4F6A516A526A536A546A40
:1000F000556A566A576A586A596A5A6A5B6A5C6AEC
:100100005D6A5E6A5F6A606B616B626B636B646B96
:10011000656B666B676B000EAA6E000EA96EA69EDD
:10012000A69CA68000000000A850116E000EAA6ECA
:10013000010EA96EA69EA69CA68000000000A850F5
:10014000126E000EAA6E020EA96EA69EA69CA68036
:1001500000000000A850136E000EAA6E030EA96ED8
:10016000A69EA69CA68000000000A850146E000E5B
:10017000AA6E040EA96EA69EA69CA6800000000092
:10018000A850156E000EAA6E050EA96EA69EA69C1E
:10019000A68000000000A850166E000EAA6E060E83
:1001A000A96EA69EA69CA68000000000A850176E0F
:1001B000000EAA6E070EA96EA69EA69CA680000041
:1001C0000000A850186E000EAA6E080EA96EA69E1A
:1001D000A69CA68000000000A850196E000EAA6E12
:1001E000090EA96EA69EA69CA68000000000A8503D
:1001F0001A6E000EAA6E0A0EA96EA69EA69CA68076
:1002000000000000A8504D6E000EAA6E0B0EA96EE5
:10021000A69EA69CA68000000000A8505F6E8B8062
:10022000E6EC36F0A7EC36F020EC35F0C00E8A6E26
:100230008C9C8C9E8C8A8C9A1FEC36F03F0E8A6EBA
:100240008C9C8C9E8C8A8C9A42EC36F08B8A23ECA8
:1002500035F0CCEC42F05FEC36F0B9EC37F0F0EC76
:1002600038F05D505E6E5F50606F1D504F6E4D50A8
:100270004E6E8C864DA442EF01F083A242EF01F056
:100280007FEC41F0B9EC37F09CEC39F0F0EC44F045
:100290003AEC45F080B674EF01F0070E5B5CD8B421
:1002A00055EF01F05B2A76EF01F05B6A3EB676EF20
:1002B00001F01550380B5C6E380E5C5CD8B465EFFD
:1002C00001F0080E5C2667EF01F0000E5C6E155021
:1002D000C70B156E5C5015124DB29CEC41F05FECF3
:1002E00036F03E8676EF01F03E965B6A80B4A0EF72
:1002F00001F0070E5A5CD8B481EF01F05A2AA2EF40
:1003000001F05A6A3EB4A2EF01F01550380B5C6E52
:10031000000E5C5CD8B491EF01F0080E5C5E93EFC8
:1003200001F0380E5C6E1550C70B156E5C5015123F
:100330004DB29CEC41F05FEC36F03E84A2EF01F050
:100340003E945A6A4DB47AEC41F03AEC45F080B2F2
:10035000C4EF01F0070E595CD8B4B2EF01F0592A8E
:10036000C6EF01F0596A3EB2C6EF01F0050E415CDE
:10037000D8B4BEEF01F0412ABFEF01F0416A42EC70
:1003800036F03E82C6EF01F03E92596A3AEC45F0F3
:10039000000E415CD8B4E8EF01F0010E415CD8B426
:1003A000E3EF0AF0020E415CD8B41BEF11F0030E2C
:1003B000415CD8B464EF20F0040E415CD8B4E3EFA4
:1003C00029F0050E415CD8B493EF2FF042EF01F015
:1003D0001AEC35F0410E26EC35F0B80E3FEC35F056
:1003E000700E58EC35F0100E58EC35F0100E58EC3D
:1003F00035F0100E58EC35F0000E58EC35F05EEC90
:1004000052F0000E58EC35F08EEC51F0000E58EC26
:1004100035F06EEC51F0000E58EC35F08EEC51F0EA
:10042000000E58EC35F0CEEC51F0000E58EC35F0E3
:100430009EEC52F0000E58EC35F08EEC51F0000EB0
:1004400058EC35F05EEC52F08EEC54F06EEC52F05D
:100450001DEC35F0400E26EC35F0B80E3FEC35F0D3
:100460007EEC52F0000E58EC35F04EEC51F0000EE0
:1004700058EC35F07EEC52F0000E58EC35F08EEC76
:1004800052F0000E58EC35F06EEC52F0000E58ECC5
:1004900035F0082A210E085CD8B454EF02F0100E93
:1004A00058EC35F049EF02F0086A700E58EC35F060
:1004B0003AEC45F01AEC35F0400E26EC35F0BA0E69
:1004C0003FEC35F01DA881EF02F08EEC54F08EEC7D
:1004D00054F08EEC54F08EEC54F0000E58EC35F0E5
:1004E0008EEC54F0000E58EC35F08EEC54F0000E0B
:1004F00058EC35F08EEC54F0000E58EC35F0ABEFC4
:1005000002F01BA4CDEF02F0FF0E58EC35F0BEEC6C
:1005100053F0FF0E58EC35F0CEEC53F0FF0E58ECD4
:1005200035F0FF0E58EC35F0FF0E58EC35F00EECC0
:1005300054F0FF0E58EC35F00EEC53F0FF0E58EC73
:1005400035F0AEEC53F0FF0E58EC35F00EEC54F0F5
:10055000FF0E58EC35F0082A1A0E085CD8B4B6EF36
:1005600002F0000E58EC35F0ABEF02F0086A1DEC1B
:1005700035F0400E26EC35F0BA0E3FEC35F0082A87
:10058000070E085CD8B4CAEF02F0000E58EC35F044
:10059000BFEF02F0086A54EF03F0FF0E58EC35F09D
:1005A0000EEC54F0FF0E58EC35F00EEC53F0FF0E4D
:1005B00058EC35F0AEEC53F0FF0E58EC35F00EEC85
:1005C00054F0FF0E58EC35F0000E58EC35F0000EEC
:1005D00058EC35F01BA21DEF03F0FF0E58EC35F080
:1005E000CEEC53F0FF0E58EC35F0FEEC53F0FF0E5E
:1005F00058EC35F06EEC53F0FF0E58EC35F04EEC45
:1006000053F0FF0E58EC35F0BEEC53F0FF0E58ECF3
:1006100035F0EEEC52F0FF0E58EC35F01DEC35F0F5
:10062000400E26EC35F0BA0E3FEC35F09EEC53F060
:10063000FF0E58EC35F054EF03F0FF0E58EC35F098
:100640000EEC53F0FF0E58EC35F0CEEC53F0FF0EED
:1006500058EC35F0DEEC53F0FF0E58EC35F06EEC54
:1006600054F0FF0E58EC35F0082A0D0E085CD8B493
:100670003FEF03F0000E58EC35F034EF03F0086A5A
:100680001DEC35F0400E26EC35F0BA0E3FEC35F09F
:10069000082A070E085CD8B453EF03F0000E58EC9C
:1006A00035F048EF03F0086A1DEC35F0480E26ECF3
:1006B00035F0BA0E3FEC35F01DB876EF03F01BA60F
:1006C00076EF03F0FF0E58EC35F0DEEC53F0FF0E42
:1006D00058EC35F0FEEC53F0FF0E58EC35F0CEEC54
:1006E00053F0FF0E58EC35F082EF03F0082A140E99
:1006F000085CD8B481EF03F0000E58EC35F076EFCB
:1007000003F0086A1DEC35F05D0E26EC35F0BA0EEC
:100710003FEC35F01DB8A9EF03F01BB0A9EF03F0D3
:10072000FF0E58EC35F02EEC53F0FF0E58EC35F080
:10073000AEEC53F0FF0E58EC35F0DEEC53F0FF0E4C
:1007400058EC35F05EEC53F0FF0E58EC35F0B5EF99
:1007500003F0082A1A0E085CD8B4B4EF03F0000EB8
:1007600058EC35F0A9EF03F0086A1AEC35F0400EAA
:1007700026EC35F0B90E3FEC35F01DB834EF05F03E
:100780001CB6CEEF03F01CB8FCEF03F01CBA2AEF46
:1007900004F01CBC5AEF04F034EF05F0FF0E58ECE7
:1007A00035F01EEC53F0FF0E58EC35F01EEC54F013
:1007B000FF0E58EC35F00EEC54F0FF0E58EC35F00F
:1007C000FF0E58EC35F0FF0E0EEC53F0FF0E58EC18
:1007D00035F01EEC53F0FF0E58EC35F0082A110EE0
:1007E000085CD8B4F9EF03F0000E58EC35F0EEEFEA
:1007F00003F0086A40EF05F0FF0E58EC35F01EECF0
:1008000053F0FF0E58EC35F01EEC54F0FF0E58EC90
:1008100035F00EEC54F0FF0E58EC35F0FF0E58ECAE
:1008200035F0FF0E9EEC53F0FF0E58EC35F01EEC49
:1008300053F0FF0E58EC35F0082A110E085CD8B4BE
:1008400027EF04F0000E58EC35F01CEF04F0086AB6
:1008500040EF05F0FF0E58EC35F06EEC53F0FF0E54
:1008600058EC35F02EEC53F0FF0E58EC35F00EEC52
:1008700053F0FF0E58EC35F06EEC4FF0FF0E58ECD5
:1008800035F01EEC4FF0FF0E58EC35F09EEC4FF0BB
:10089000FF0E58EC35F03EEC4FF0FF0E58EC35F003
:1008A0007EEC4FF0FF0E58EC35F0000E58EC35F0B2
:1008B00040EF05F0FF0E58EC35F0DEEC53F0FF0E84
:1008C00058EC35F00EEC53F0FF0E58EC35F0AEEC72
:1008D00053F0FF0E58EC35F0000E58EC35F02B506D
:1008E000536E539E010E535CD8B494EF04F0490E3E
:1008F000535CD8B4BCEF04F0030E535CD8B4E4EFFF
:1009000004F0430E535CD8B40CEF05F0082A1E0E19
:10091000085CD8B491EF04F0000E58EC35F086EF87
:1009200004F0086A40EF05F0000E58EC35F0FF0EB9
:1009300058EC35F00EEC53F0FF0E58EC35F01EEC91
:1009400053F0FF0E58EC35F08EEC54F0000E58ECDE
:1009500035F08EEC54F0000E58EC35F0000E58ECEB
:1009600035F0000E58EC35F0000E58EC35F0000E66
:1009700058EC35F040EF05F0000E58EC35F0FF0E66
:1009800058EC35F0AEEC53F0FF0E58EC35F01EECA1
:1009900053F0FF0E58EC35F08EEC54F0000E58EC8E
:1009A00035F08EEC54F0000E58EC35F0000E58EC9B
:1009B00035F0000E58EC35F0000E58EC35F0000E16
:1009C00058EC35F040EF05F0000E58EC35F0FF0E16
:1009D00058EC35F01EEC53F0FF0E58EC35F0EEEC11
:1009E00052F0FF0E58EC35F01EEC54F0FF0E58ECB0
:1009F00035F08EEC54F0000E58EC35F0000E58EC4B
:100A000035F0000E58EC35F0000E58EC35F0000EC5
:100A100058EC35F040EF05F0000E58EC35F0FF0EC5
:100A200058EC35F01EEC53F0FF0E58EC35F00EECA0
:100A300053F0FF0E58EC35F00EEC53F0FF0E58EC6F
:100A400035F08EEC54F0000E58EC35F0000E58ECFA
:100A500035F0000E58EC35F0000E58EC35F0000E75
:100A600058EC35F040EF05F0082A320E085CD8B497
:100A70003FEF05F0000E58EC35F034EF05F0086A52
:100A80001AEC35F0730E26EC35F0B90E3FEC35F06C
:100A90001DB87EEF05F01CA27EEF05F0FF0E58ECAE
:100AA00035F00EEC54F0FF0E58EC35F06EEC53F0D0
:100AB000FF0E58EC35F01DEC35F0400E26EC35F00D
:100AC000B90E3FEC35F09EEC53F0FF0E58EC35F0CC
:100AD0002EEC53F0FF0E58EC35F0BEEC53F0FF0E49
:100AE00058EC35F00EEC53F0FF0E58EC35F02EECD0
:100AF00053F0FF0E58EC35F09EEF05F0082A0E0E6D
:100B0000085CD8B489EF05F0000E58EC35F07EEFA4
:100B100005F0086A1DEC35F0400E26EC35F0B90EF4
:100B20003FEC35F0082A1F0E085CD8B49DEF05F0A5
:100B3000000E58EC35F092EF05F0086A1DEC35F028
:100B4000600E26EC35F0B90E3FEC35F01DB8CEEF57
:100B500005F01CA0CEEF05F0FF0E58EC35F05EEC72
:100B600053F0FF0E58EC35F06EEC53F0FF0E58ECDE
:100B700035F0FF0E58EC35F0FF0E58EC35F03EEC3A
:100B800053F0FF0E58EC35F00EEC54F0FF0E58EC1D
:100B900035F0000E58EC35F0DAEF05F0082A1C0E9F
:100BA000085CD8B4D9EF05F0000E58EC35F0CEEF64
:100BB00005F0086A1AEC35F0400E26EC35F0BB0E55
:100BC0003FEC35F04DB0EAEF05F01D504F6E506A26
:100BD000FFEF05F01D504F5CD8A43F9A000E505C0B
:100BE000D8A4F5EF05F01D504F6E3FBAFFEF05F0AA
:100BF000000E4F5CD8B4FFEF05F044EC46F0000E59
:100C00004F5CD8A408EF06F0C2EC46F052EF06F0B5
:100C1000400E4F5CD8A411EF06F0E2EC46F052EF24
:100C200006F0200E4F5CD8A41AEF06F003EC47F054
:100C300052EF06F0100E4F5CD8A423EF06F024EC20
:100C400047F052EF06F0080E4F5CD8A42CEF06F0E8
:100C50005CEC47F052EF06F0020E4F5CD8A435EF83
:100C600006F0AAEC47F052EF06F0010E4F5CD8A454
:100C70003EEF06F0F8EC47F052EF06F0FF0E58ECAE
:100C800035F078EC48F04F5075EC45F0FF0E58EC1D
:100C900035F0FF0E58EC35F0D7EC45F08EEC54F003
:100CA0008EEC54F01AEC35F0400E26EC35F0BD0E0B
:100CB0003FEC35F0000E58EC35F09EEC51F0000E94
:100CC00058EC35F06EEC52F0000E58EC35F0280E72
:100CD00058EC35F0280E58EC35F0280E58EC35F06D
:100CE000280E58EC35F0280E58EC35F0000E58EC74
:100CF00035F01AEC35F0530E26EC35F0BD0E3FEC16
:100D000035F0010E625DD8A4A5EF06F0000E58EC98
:100D100035F08EEC54F0000E58EC35F08EEC54F0BB
:100D2000000E58EC35F0000E58EC35F0000E58EC83
:100D300035F09EEC4EF0000E58EC35F08EEC4EF097
:100D4000000E58EC35F0CEEF07F0020E625DD8A42D
:100D5000C9EF06F0000E58EC35F08EEC54F0000EA2
:100D600058EC35F0AEEC4EF0000E58EC35F0AEEC31
:100D70004EF0000E58EC35F0400E58EC35F0000EF9
:100D800058EC35F07EEC4EF0000E58EC35F0CEEF1E
:100D900007F0030E625DD8A4EDEF06F0000E58ECEC
:100DA00035F08EEC54F0000E58EC35F08EEC54F02B
:100DB000000E58EC35F0000E58EC35F0000E58ECF3
:100DC00035F0AEEC4EF0000E58EC35F0EEEC4EF097
:100DD000000E58EC35F0CEEF07F0040E625DD8A49B
:100DE00011EF07F0000E58EC35F08EEC54F0FF0ECA
:100DF00058EC35F08EEC4FF0FF0E58EC35F08EECE1
:100E00004FF0FF0E58EC35F0BF0E58EC35F0FF0EEA
:100E100058EC35F02EEC4FF0FF0E58EC35F0CEEFDD
:100E200007F0050E625DD8A435EF07F0000E58EC10
:100E300035F08EEC54F0000E58EC35F08EEC54F09A
:100E4000000E58EC35F0000E58EC35F0FF0E58EC63
:100E500035F09EEC4FF0FF0E58EC35F06EEC4FF095
:100E6000FF0E58EC35F0CEEF07F0060E625DD8A409
:100E700059EF07F0FF0E58EC35F01EEC4FF0FF0E67
:100E800058EC35F07EEC4FF0FF0E58EC35F06EEC80
:100E90004FF0FF0E58EC35F0BF0E58EC35F0FF0E5A
:100EA00058EC35F04EEC4FF0FF0E58EC35F0CEEF2D
:100EB00007F0070E625DD8A47DEF07F0000E58EC36
:100EC00035F08EEC54F0000E58EC35F0000E58EC76
:100ED00035F0FF0E58EC35F01EEC4FF0FF0E58ECDD
:100EE00035F09EEC4FF0FF0E58EC35F02EEC4FF045
:100EF000FF0E58EC35F0CEEF07F0000E58EC35F051
:100F0000100E58EC35F0100E58EC35F0100E58EC71
:100F100035F0100E58EC35F0100E58EC35F0000E90
:100F200058EC35F0100E58EC35F0100E58EC35F04A
:100F3000100E58EC35F0100E58EC35F0100E58EC41
:100F400035F0000E58EC35F0100E58EC35F0100E60
:100F500058EC35F0100E58EC35F0100E58EC35F01A
:100F6000100E58EC35F0000E58EC35F0400E58ECF1
:100F700035F0000E58EC35F0100E58EC35F0100E30
:100F800058EC35F0100E58EC35F0100E58EC35F0EA
:100F9000100E58EC35F0000E58EC35F0000E58EC01
:100FA00035F0EEEC51F0000E58EC35F0BEEC51F09F
:100FB000000E58EC35F0DEEC52F0000E58EC35F037
:100FC0001AEC35F0400E26EC35F0BC0E3FEC35F057
:100FD000000E58EC35F0CEEC51F0000E58EC35F028
:100FE0001EEC52F0000E58EC35F0280E58EC35F09F
:100FF000280E58EC35F0280E58EC35F0280E58EC39
:1010000035F0280E58EC35F0000E58EC35F01AEC9F
:1010100035F0530E26EC35F0BC0E3FEC35F0155094
:10102000380B406E000E405CD8A43FEF08F0000E75
:1010300058EC35F05EEC52F0000E58EC35F0BEEC9A
:1010400052F0000E58EC35F03EEC52F0000E58EC29
:1010500035F06EEC4EF0000E58EC35F08EEC54F09E
:10106000000E58EC35F08EEC54F0000E58EC35F0D4
:101070008EEC54F0000E58EC35F08AEF09F0080EB3
:10108000405CD8A46CEF08F0000E58EC35F05EEC34
:1010900052F0000E58EC35F0BEEC52F0000E58EC59
:1010A00035F03EEC52F0000E58EC35F07EEC4EF090
:1010B000000E58EC35F08EEC54F0000E58EC35F084
:1010C0008EEC54F0000E58EC35F08EEC54F0000E1F
:1010D00058EC35F08AEF09F0100E405CD8A499EF77
:1010E00008F0000E58EC35F05EEC52F0000E58ECB3
:1010F00035F0BEEC52F0000E58EC35F03EEC52F0FC
:10110000000E58EC35F08EEC4EF0000E58EC35F039
:101110008EEC54F0000E58EC35F08EEC54F0000ECE
:1011200058EC35F08EEC54F0000E58EC35F08AEFA8
:1011300009F0180E405CD8A4DDEF08F0000E58EC62
:1011400035F08EEC52F0000E58EC35F06EEC52F0AB
:10115000000E58EC35F05EEC51F0000E58EC35F016
:101160008EEC54F083A2C9EF08F0FF0E58EC35F076
:10117000EEEC52F0FF0E58EC35F00EEC53F0FF0E93
:1011800058EC35F01EEC54F0FF0E58EC35F08AEFB9
:1011900009F0000E58EC35F06EEC52F0000E58ECF1
:1011A00035F03EEC52F0000E58EC35F07EEC51F08C
:1011B000000E58EC35F08AEF09F0200E405CD8A400
:1011C0000AEF09F0000E58EC35F05EEC52F0000E1C
:1011D00058EC35F0BEEC52F0000E58EC35F03EEC19
:1011E00052F0000E58EC35F0AEEC4EF0000E58EC1C
:1011F00035F08EEC54F0000E58EC35F08EEC54F0D7
:10120000000E58EC35F08EEC54F0000E58EC35F032
:101210008AEF09F0280E405CD8A437EF09F0000EE1
:1012200058EC35F05EEC52F0000E58EC35F0BEECA8
:1012300052F0000E58EC35F03EEC52F0000E58EC37
:1012400035F0BEEC4EF0000E58EC35F08EEC54F05C
:10125000000E58EC35F08EEC54F0000E58EC35F0E2
:101260008EEC54F0000E58EC35F08AEF09F0300E99
:10127000405CD8A464EF09F0000E58EC35F05EEC49
:1012800052F0000E58EC35F0BEEC52F0000E58EC67
:1012900035F03EEC52F0000E58EC35F0CEEC4EF04E
:1012A000000E58EC35F08EEC54F0000E58EC35F092
:1012B0008EEC54F0000E58EC35F08EEC54F0000E2D
:1012C00058EC35F08AEF09F0000E58EC35F05EEC82
:1012D00052F0000E58EC35F0BEEC52F0000E58EC17
:1012E00035F03EEC52F0000E58EC35F0DEEC4EF0EE
:1012F000000E58EC35F08EEC54F0000E58EC35F042
:101300008EEC54F0000E58EC35F08EEC54F0000EDC
:1013100058EC35F01DA851921DB8A5EF09F0020E4A
:101320001F5CD8B4B1EF09F0030E1F5CD8B4B1EF65
:1013300009F0010E1F5CD8B4B1EF09F0210E1F5C5B
:10134000D8B4B1EF09F0ABEF09F051B2ABEF09F04F
:101350005FEC36F05182206A216A226A236A266A8B
:10136000276A205093EC45F01AEC35F0400E26EC3D
:1013700035F0BE0E3FEC35F0080E58EC35F0F80EA7
:1013800058EC35F0080E58EC35F0E00E58EC35F01E
:10139000200E58EC35F0000E58EC35F0000E58ECED
:1013A00035F0059CAFEC45F0215093EC45F01AEC7C
:1013B00035F05A0E26EC35F0BE0E3FEC35F0F80E47
:1013C00058EC35F0000E58EC35F0E00E58EC35F0E6
:1013D000200E58EC35F0E00E58EC35F0000E58ECCD
:1013E00035F0000E58EC35F0059CAFEC45F022507E
:1013F00093EC45F01AEC35F0400E26EC35F0BF0EBC
:101400003FEC35F0059CAFEC45F0AEEC54F02350CA
:1014100093EC45F01AEC35F04E0E26EC35F0BF0E8D
:101420003FEC35F0059CAFEC45F0265093EC45F0D1
:101430001AEC35F05C0E26EC35F0BF0E3FEC35F0C3
:10144000059CAFEC45F0AEEC54F0275093EC45F022
:101450001AEC35F06A0E26EC35F0BF0E3FEC35F095
:10146000059CAFEC45F01DEC35F0460E26EC35F052
:10147000BC0E3FEC35F0700E58EC35F0100E58EC09
:1014800035F0100E58EC35F0100E58EC35F0000E1B
:1014900058EC35F0AEEC51F0000E58EC35F03EEC67
:1014A00052F0000E58EC35F02EEC52F0000E58ECD5
:1014B00035F0082A220E085CD8B464EF0AF0100E4A
:1014C00058EC35F059EF0AF0086A700E58EC35F018
:1014D0001DEC35F0460E26EC35F0BD0E3FEC35F038
:1014E000000E58EC35F06EEC4EF0000E58EC35F076
:1014F000280E58EC35F0280E58EC35F0280E58EC34
:1015000035F0280E58EC35F0280E58EC35F0000E6A
:1015100058EC35F013500F0B406E30EC3AF01DECE8
:1015200035F0460E26EC35F0BE0E3FEC35F0000EE1
:1015300058EC35F07EEC4EF0000E58EC35F0280EED
:1015400058EC35F0280E58EC35F0280E58EC35F0F4
:10155000280E58EC35F0280E58EC35F0000E58ECFB
:1015600035F01450F00B406E404240424042404241
:1015700030EC3AF01DEC35F0460E26EC35F0BF0E9F
:101580003FEC35F0000E58EC35F08EEC4EF0000ECE
:1015900058EC35F0280E58EC35F0280E58EC35F0A4
:1015A000280E58EC35F0280E58EC35F0280E58EC83
:1015B00035F0000E58EC35F014500F0B406E30EC47
:1015C0003AF042EF01F0506A1AEC35F0410E26EC89
:1015D00035F0B80E3FEC35F0700E58EC35F0100ECB
:1015E00058EC35F0100E58EC35F0100E58EC35F084
:1015F000000E58EC35F06EEC51F0000E58EC35F062
:101600006EEC52F0000E58EC35F0EEEC4EF0000EA1
:1016100058EC35F0AEEC4EF0000E58EC35F07EECA8
:101620004EF0000E58EC35F0CEEC4EF0000E58ECBB
:1016300035F08EEC54F05EEC52F0000E58EC35F0C4
:101640008EEC51F0000E58EC35F0AEEC51F01DEC84
:1016500035F0400E26EC35F0B80E3FEC35F0000EBC
:1016600058EC35F0CEEC51F0000E58EC35F06EEC45
:1016700052F0000E58EC35F07EEC52F0000E58ECB3
:1016800035F08EEC51F0000E58EC35F05EEC52F077
:10169000000E58EC35F0082A200E085CD8B456EF3E
:1016A0000BF0100E58EC35F04BEF0BF0086A700E93
:1016B00058EC35F01AEC35F0410E26EC35F0B90E49
:1016C0003FEC35F0FF0E58EC35F0EEEC52F0FF0E2B
:1016D00058EC35F01EEC53F0FF0E58EC35F01EECD4
:1016E00053F0FF0E58EC35F0FEEC53F0FF0E58ECC3
:1016F00035F02EEC53F0FF0E58EC35F00EEC54F0B4
:10170000FF0E58EC35F00EEC54F0FF0E58EC35F0AF
:101710001DEC35F0410E26EC35F0B90E3FEC35F0FE
:10172000FF0E58EC35F01EEC53F0FF0E58EC35F080
:10173000EEEC52F0FF0E58EC35F01EEC54F0FF0EBC
:1017400058EC35F0EEEC52F0FF0E58EC35F080B06E
:10175000C4EF0BF0070E565CD8B4B2EF0BF0562A6C
:10176000C6EF0BF0566A3EB0C6EF0BF0060E425CB9
:10177000D8B4BEEF0BF0422ABFEF0BF0426A42EC46
:1017800036F03E80C6EF0BF03E90566A84B6E4EF2A
:101790000BF0070E555CD8B4D1EF0BF0552AE6EFED
:1017A0000BF0556A3EBCE6EF0BF0000E425CD8B47D
:1017B000DDEF0BF04206DFEF0BF0060E426E42EC5F
:1017C00036F03E8CE6EF0BF03E9C556A3AEC45F065
:1017D0001AEC35F0410E26EC35F0BA0E3FEC35F040
:1017E000000E425CD8B415EF0CF0010E425CD8B488
:1017F000DBEF0CF0020E425CD8B4A1EF0DF0030E4B
:10180000425CD8B467EF0EF0040E425CD8B42DEF02
:101810000FF0050E425CD8B4F3EF0FF0060E425CF9
:10182000D8B4B9EF10F017EF11F06EEC4EF0000ED7
:1018300058EC35F06EEC4EF0000E58EC35F0BEEC86
:1018400051F0000E58EC35F01DEC35F0410E26EC51
:1018500035F0BA0E3FEC35F01150EDEC45F01AECD6
:1018600035F0410E26EC35F0BB0E3FEC35F06EEC5A
:101870004EF0000E58EC35F07EEC4EF0000E58ECB9
:1018800035F0BEEC51F0000E58EC35F01DEC35F0A3
:10189000410E26EC35F0BB0E3FEC35F01250EDEC6E
:1018A00045F01AEC35F0410E26EC35F0BC0E3FEC5D
:1018B00035F06EEC4EF0000E58EC35F08EEC4EF03C
:1018C000000E58EC35F0BEEC51F0000E58EC35F03F
:1018D0001DEC35F0410E26EC35F0BC0E3FEC35F03A
:1018E0001350EDEC45F01AEC35F0410E26EC35F0D6
:1018F000BD0E3FEC35F06EEC4EF0000E58EC35F0BE
:101900009EEC4EF0000E58EC35F0BEEC51F0000E9F
:1019100058EC35F01DEC35F0410E26EC35F0BD0EDF
:101920003FEC35F01450EDEC45F01AEC35F0410E7B
:1019300026EC35F0BE0E3FEC35F06EEC4EF0000EAE
:1019400058EC35F0AEEC4EF0000E58EC35F0BEEC35
:1019500051F0000E58EC35F01DEC35F0410E26EC40
:1019600035F0BE0E3FEC35F01550EDEC45F01AECBD
:1019700035F0410E26EC35F0BF0E3FEC35F06EEC45
:101980004EF0000E58EC35F0BEEC4EF0000E58EC68
:1019900035F0BEEC51F0000E58EC35F01DEC35F092
:1019A000410E26EC35F0BF0E3FEC35F01650EDEC55
:1019B00045F017EF11F06EEC4EF0000E58EC35F0DC
:1019C000CEEC4EF0000E58EC35F0BEEC51F0000EAF
:1019D00058EC35F01DEC35F0410E26EC35F0BA0E22
:1019E0003FEC35F01750EDEC45F01AEC35F0410EB8
:1019F00026EC35F0BB0E3FEC35F06EEC4EF0000EF1
:101A000058EC35F0DEEC4EF0000E58EC35F0BEEC44
:101A100051F0000E58EC35F01DEC35F0410E26EC7F
:101A200035F0BB0E3FEC35F01850EDEC45F01AECFC
:101A300035F0410E26EC35F0BC0E3FEC35F06EEC87
:101A40004EF0000E58EC35F0EEEC4EF0000E58EC77
:101A500035F0BEEC51F0000E58EC35F01DEC35F0D1
:101A6000410E26EC35F0BC0E3FEC35F01950EDEC94
:101A700045F01AEC35F0410E26EC35F0BD0E3FEC8A
:101A800035F06EEC4EF0000E58EC35F0FEEC4EF0FA
:101A9000000E58EC35F0BEEC51F0000E58EC35F06D
:101AA0001DEC35F0410E26EC35F0BD0E3FEC35F067
:101AB0001A50EDEC45F01AEC35F0410E26EC35F0FD
:101AC000BE0E3FEC35F06EEC4EF0000E58EC35F0EB
:101AD0004EEC51F0000E58EC35F0BEEC51F0000E1B
:101AE00058EC35F01DEC35F0410E26EC35F0BE0E0D
:101AF0003FEC35F01B50EDEC45F01AEC35F0410EA3
:101B000026EC35F0BF0E3FEC35F06EEC4EF0000EDB
:101B100058EC35F05EEC51F0000E58EC35F0BEECB0
:101B200051F0000E58EC35F01DEC35F0410E26EC6E
:101B300035F0BF0E3FEC35F01C50EDEC45F017EFE3
:101B400011F06EEC4EF0000E58EC35F06EEC51F0EA
:101B5000000E58EC35F0BEEC51F0000E58EC35F0AC
:101B60001DEC35F0410E26EC35F0BA0E3FEC35F0A9
:101B70001D50EDEC45F01AEC35F0410E26EC35F039
:101B8000BB0E3FEC35F06EEC4EF0000E58EC35F02D
:101B90007EEC51F0000E58EC35F0BEEC51F0000E2A
:101BA00058EC35F01DEC35F0410E26EC35F0BB0E4F
:101BB0003FEC35F01E50EDEC45F01AEC35F0410EDF
:101BC00026EC35F0BC0E3FEC35F06EEC4EF0000E1E
:101BD00058EC35F08EEC51F0000E58EC35F0BEECC0
:101BE00051F0000E58EC35F01DEC35F0410E26ECAE
:101BF00035F0BC0E3FEC35F01F50EDEC45F01AEC23
:101C000035F0410E26EC35F0BD0E3FEC35F06EECB4
:101C10004EF0000E58EC35F09EEC51F0000E58ECF2
:101C200035F0BEEC51F0000E58EC35F01DEC35F0FF
:101C3000410E26EC35F0BD0E3FEC35F02050EDECBA
:101C400045F01AEC35F0410E26EC35F0BE0E3FECB7
:101C500035F07EEC4EF0000E58EC35F06EEC4EF0A8
:101C6000000E58EC35F0BEEC51F0000E58EC35F09B
:101C70001DEC35F0410E26EC35F0BE0E3FEC35F094
:101C80002150EDEC45F01AEC35F0410E26EC35F024
:101C9000BF0E3FEC35F07EEC4EF0000E58EC35F008
:101CA0007EEC4EF0000E58EC35F0BEEC51F0000E1C
:101CB00058EC35F01DEC35F0410E26EC35F0BF0E3A
:101CC0003FEC35F02250EDEC45F017EF11F07EECD3
:101CD0004EF0000E58EC35F08EEC4EF0000E58EC45
:101CE00035F0BEEC51F0000E58EC35F01DEC35F03F
:101CF000410E26EC35F0BA0E3FEC35F02350EDECFA
:101D000045F01AEC35F0410E26EC35F0BB0E3FECF9
:101D100035F07EEC4EF0000E58EC35F09EEC4EF0B7
:101D2000000E58EC35F0BEEC51F0000E58EC35F0DA
:101D30001DEC35F0410E26EC35F0BB0E3FEC35F0D6
:101D40002450EDEC45F01AEC35F0410E26EC35F060
:101D5000BC0E3FEC35F07EEC4EF0000E58EC35F04A
:101D6000AEEC4EF0000E58EC35F0BEEC51F0000E2B
:101D700058EC35F01DEC35F0410E26EC35F0BC0E7C
:101D80003FEC35F02550EDEC45F01AEC35F0410E06
:101D900026EC35F0BD0E3FEC35F07EEC4EF0000E3B
:101DA00058EC35F0BEEC4EF0000E58EC35F0BEECC1
:101DB00051F0000E58EC35F01DEC35F0410E26ECDC
:101DC00035F0BD0E3FEC35F02650EDEC45F01AEC49
:101DD00035F0410E26EC35F0BE0E3FEC35F07EECD2
:101DE0004EF0000E58EC35F0CEEC4EF0000E58ECF4
:101DF00035F0BEEC51F0000E58EC35F01DEC35F02E
:101E0000410E26EC35F0BE0E3FEC35F02750EDECE0
:101E100045F01AEC35F0410E26EC35F0BF0E3FECE4
:101E200035F07EEC4EF0000E58EC35F0DEEC4EF066
:101E3000000E58EC35F0BEEC51F0000E58EC35F0C9
:101E40001DEC35F0410E26EC35F0BF0E3FEC35F0C1
:101E50002850EDEC45F017EF11F07EEC4EF0000E3F
:101E600058EC35F0EEEC4EF0000E58EC35F0BEECD0
:101E700051F0000E58EC35F01DEC35F0410E26EC1B
:101E800035F0BA0E3FEC35F02950EDEC45F01AEC88
:101E900035F0410E26EC35F0BB0E3FEC35F07EEC14
:101EA0004EF0000E58EC35F0FEEC4EF0000E58EC03
:101EB00035F0BEEC51F0000E58EC35F01DEC35F06D
:101EC000410E26EC35F0BB0E3FEC35F02A50EDEC20
:101ED00045F01AEC35F0410E26EC35F0BC0E3FEC27
:101EE00035F07EEC4EF0000E58EC35F04EEC51F033
:101EF000000E58EC35F0BEEC51F0000E58EC35F009
:101F00001DEC35F0410E26EC35F0BC0E3FEC35F003
:101F10002B50EDEC45F01AEC35F0410E26EC35F087
:101F2000BD0E3FEC35F07EEC4EF0000E58EC35F077
:101F30005EEC51F0000E58EC35F0BEEC51F0000EA6
:101F400058EC35F01DEC35F0410E26EC35F0BD0EA9
:101F50003FEC35F02C50EDEC45F01AEC35F0410E2D
:101F600026EC35F0BE0E3FEC35F07EEC4EF0000E68
:101F700058EC35F06EEC51F0000E58EC35F0BEEC3C
:101F800051F0000E58EC35F01DEC35F0410E26EC0A
:101F900035F0BE0E3FEC35F02D50EDEC45F01AEC6F
:101FA00035F0410E26EC35F0BF0E3FEC35F07EECFF
:101FB0004EF0000E58EC35F07EEC51F0000E58EC6F
:101FC00035F0BEEC51F0000E58EC35F01DEC35F05C
:101FD000410E26EC35F0BF0E3FEC35F02E50EDEC07
:101FE00045F017EF11F07EEC4EF0000E58EC35F096
:101FF0008EEC51F0000E58EC35F0BEEC51F0000EB6
:1020000058EC35F01DEC35F0410E26EC35F0BA0EEB
:102010003FEC35F02F50EDEC45F01AEC35F0410E69
:1020200026EC35F0BB0E3FEC35F07EEC4EF0000EAA
:1020300058EC35F09EEC51F0000E58EC35F0BEEC4B
:1020400051F0000E58EC35F01DEC35F0410E26EC49
:1020500035F0BB0E3FEC35F03050EDEC45F01AECAE
:1020600035F0410E26EC35F0BC0E3FEC35F08EEC31
:102070004EF0000E58EC35F06EEC4EF0000E58ECC1
:1020800035F0BEEC51F0000E58EC35F01DEC35F09B
:10209000410E26EC35F0BC0E3FEC35F03150EDEC46
:1020A00045F01AEC35F0410E26EC35F0BD0E3FEC54
:1020B00035F08EEC4EF0000E58EC35F07EEC4EF024
:1020C000000E58EC35F0BEEC51F0000E58EC35F037
:1020D0001DEC35F0410E26EC35F0BD0E3FEC35F031
:1020E0003250EDEC45F01AEC35F0410E26EC35F0AF
:1020F000BE0E3FEC35F08EEC4EF0000E58EC35F095
:102100008EEC4EF0000E58EC35F0BEEC51F0000EA7
:1021100058EC35F01DEC35F0410E26EC35F0BE0ED6
:102120003FEC35F03350EDEC45F01AEC35F0410E54
:1021300026EC35F0BF0E3FEC35F08EEC4EF0000E85
:1021400058EC35F09EEC4EF0000E58EC35F0BEEC3D
:1021500051F0000E58EC35F01DEC35F0410E26EC38
:1021600035F0BF0E3FEC35F03450EDEC45F017EF95
:1021700011F08EEC4EF0000E58EC35F0AEEC4EF057
:10218000000E58EC35F0BEEC51F0000E58EC35F076
:102190001DEC35F0410E26EC35F0BA0E3FEC35F073
:1021A0003550EDEC45F01AEC35F0410E26EC35F0EB
:1021B000BB0E3FEC35F08EEC4EF0000E58EC35F0D7
:1021C000BEEC4EF0000E58EC35F0BEEC51F0000EB7
:1021D00058EC35F01DEC35F0410E26EC35F0BB0E19
:1021E0003FEC35F03650EDEC45F01AEC35F0410E91
:1021F00026EC35F0BC0E3FEC35F08EEC4EF0000EC8
:1022000058EC35F0CEEC4EF0000E58EC35F0BEEC4C
:1022100051F0000E58EC35F01DEC35F0410E26EC77
:1022200035F0BC0E3FEC35F03750EDEC45F049ECA5
:1022300039F042EF01F01AEC35F0410E26EC35F0A2
:10224000B80E3FEC35F0700E58EC35F0100E58EC2F
:1022500035F0100E58EC35F0100E58EC35F0000E3D
:1022600058EC35F06EEC51F0000E58EC35F06EEC99
:1022700052F0000E58EC35F0EEEC4EF0000E58EC3B
:1022800035F0AEEC4EF0000E58EC35F07EEC4EF032
:10229000000E58EC35F0CEEC4EF0000E58EC35F058
:1022A0008EEC54F06EEC52F0000E58EC35F08EECE3
:1022B00051F0000E58EC35F07EEC52F01DEC35F08C
:1022C000400E26EC35F0B80E3FEC35F0000E58EC21
:1022D00035F07EEC52F0000E58EC35F0CEEC51F0BB
:1022E000000E58EC35F01EEC52F0000E58EC35F0B4
:1022F000AEEC51F0000E58EC35F0082A260E085CC2
:10230000D8B488EF11F0100E58EC35F07DEF11F0D5
:10231000086A700E58EC35F03AEC45F0000E435C5C
:10232000D8B49AEF11F0010E435CD8B4DAEF14F090
:1023300042EF01F01AEC35F0460E26EC35F0B90EFE
:102340003FEC35F06EEC52F0000E58EC35F08EECB0
:1023500051F0000E58EC35F0FEEC51F0000E58EC48
:1023600035F08EEC51F0000E58EC35F06EEC51F07B
:10237000000E58EC35F07EEC52F0000E58EC35F0C3
:102380008EEC54F04EEC51F0000E58EC35F07EEC33
:1023900051F0000E58EC35F07EEC51F01DEC35F0AC
:1023A000400E26EC35F0B90E3FEC35F0000E58EC3F
:1023B00035F05EEC52F0000E58EC35F08EEC51F03A
:1023C000000E58EC35F06EEC52F0000E58EC35F083
:1023D0006EEC52F0000E58EC35F080B008EF12F0C1
:1023E000070E565CD8B4F8EF11F0562A0AEF12F037
:1023F000566A3EB00AEF12F00A0E465CD8B404EFFB
:1024000012F0462A05EF12F0466A3E800AEF12F0FB
:102410003E90566A84B626EF12F0070E555CD8B48B
:1024200015EF12F0552A28EF12F0556A3EBC28EF3E
:1024300012F0000E465CD8B421EF12F0460623EFEE
:1024400012F00A0E466E3E8C28EF12F03E9C556A42
:102450003F941AEC35F04A0E26EC35F0BB0E3FECFB
:1024600035F0000E465CD8B44AEF12F0000E58EC7E
:1024700035F06EEC4EF0000E58EC35F06EEC4EF090
:10248000000E58EC35F0BEEC51F0000E58EC35F073
:102490005CEF12F0FF0E58EC35F00EEC4FF0FF0E33
:1024A00058EC35F00EEC4FF0FF0E58EC35F05EECCA
:1024B00053F0FF0E58EC35F01AEC35F0670E26ECB1
:1024C00035F0BB0E3FEC35F0010E465CD8B47DEF25
:1024D00012F0000E58EC35F06EEC4EF0000E58EC99
:1024E00035F07EEC4EF0000E58EC35F0BEEC51F0BD
:1024F000000E58EC35F08FEF12F0FF0E58EC35F06F
:102500000EEC4FF0FF0E58EC35F01EEC4FF0FF0EC6
:1025100058EC35F05EEC53F0FF0E58EC35F01DEC46
:1025200035F0440E26EC35F0BB0E3FEC35F0020ED4
:10253000465CD8B4B0EF12F0000E58EC35F06EECFB
:102540004EF0000E58EC35F08EEC4EF0000E58ECCC
:1025500035F0BEEC51F0000E58EC35F0C2EF12F041
:10256000FF0E58EC35F00EEC4FF0FF0E58EC35F046
:102570002EEC4FF0FF0E58EC35F05EEC53F0FF0EF2
:1025800058EC35F01DEC35F0610E26EC35F0BB0E45
:102590003FEC35F0030E465CD8B4E3EF12F0000ECA
:1025A00058EC35F06EEC4EF0000E58EC35F09EEC29
:1025B0004EF0000E58EC35F0BEEC51F0000E58EC29
:1025C00035F0F5EF12F0FF0E58EC35F00EEC4FF051
:1025D000FF0E58EC35F03EEC4FF0FF0E58EC35F0A6
:1025E0005EEC53F0FF0E58EC35F01AEC35F04A0E65
:1025F00026EC35F0BC0E3FEC35F0040E465CD8B44A
:1026000016EF13F0000E58EC35F06EEC4EF0000EA5
:1026100058EC35F0AEEC4EF0000E58EC35F0BEEC58
:1026200051F0000E58EC35F028EF13F0FF0E58EC87
:1026300035F00EEC4FF0FF0E58EC35F04EEC4FF04D
:10264000FF0E58EC35F05EEC53F0FF0E58EC35F011
:102650001AEC35F0670E26EC35F0BC0E3FEC35F089
:10266000050E465CD8B449EF13F0000E58EC35F077
:102670006EEC4EF0000E58EC35F0BEEC4EF0000E55
:1026800058EC35F0BEEC51F0000E58EC35F05BEF35
:1026900013F0FF0E58EC35F00EEC4FF0FF0E58EC37
:1026A00035F05EEC4FF0FF0E58EC35F05EEC53F079
:1026B000FF0E58EC35F01DEC35F0440E26EC35F0ED
:1026C000BC0E3FEC35F0060E465CD8B47CEF13F040
:1026D000000E58EC35F06EEC4EF0000E58EC35F074
:1026E000CEEC4EF0000E58EC35F0BEEC51F0000E82
:1026F00058EC35F08EEF13F0FF0E58EC35F00EEC81
:102700004FF0FF0E58EC35F06EEC4FF0FF0E58EC2A
:1027100035F05EEC53F0FF0E58EC35F01DEC35F063
:10272000610E26EC35F0B40E3FEC35F0070E465C3A
:10273000D8B4AFEF13F0000E58EC35F06EEC4EF05D
:10274000000E58EC35F0DEEC4EF0000E58EC35F093
:10275000BEEC51F0000E58EC35F0C1EF13F0FF0E57
:1027600058EC35F00EEC4FF0FF0E58EC35F07EECE7
:102770004FF0FF0E58EC35F05EEC53F0FF0E58ECC6
:1027800035F01AEC35F04A0E26EC35F0BD0E3FEC74
:1027900035F0080E465CD8B4E2EF13F0000E58ECAA
:1027A00035F06EEC4EF0000E58EC35F0EEEC4EF0DD
:1027B000000E58EC35F0BEEC51F0000E58EC35F040
:1027C000F4EF13F0FF0E58EC35F00EEC4FF0FF0E67
:1027D00058EC35F08EEC4FF0FF0E58EC35F05EEC17
:1027E00053F0FF0E58EC35F01AEC35F0670E26EC7E
:1027F00035F0BD0E3FEC35F0090E465CD8B415EF50
:1028000014F0000E58EC35F06EEC4EF0000E58EC63
:1028100035F0FEEC4EF0000E58EC35F0BEEC51F009
:10282000000E58EC35F027EF14F0FF0E58EC35F0A1
:102830000EEC4FF0FF0E58EC35F09EEC4FF0FF0E13
:1028400058EC35F05EEC53F0FF0E58EC35F01AEC16
:1028500035F04A0E26EC35F0BF0E3FEC35F00A0E8F
:10286000465CD8B47AEF14F0000E58EC35F07EECEC
:1028700051F0000E58EC35F08EEC51F0000E58EC93
:1028800035F09EEC51F0000E58EC35F04EEC51F066
:10289000000E58EC35F08EEC52F0000E58EC35F08E
:1028A000FEEC51F0000E58EC35F07EEC52F0000ECC
:1028B00058EC35F08EEC54F0FEEC51F0000E58EC74
:1028C00035F01DEC35F0400E26EC35F0BF0E3FEC38
:1028D00035F02EEC52F0000E58EC35F04EEC51F085
:1028E000000E58EC35F07EEC51F0000E58EC35F04F
:1028F000BEEF14F0FF0E58EC35F01EEC53F0FF0E57
:1029000058EC35F02EEC53F0FF0E58EC35F03EEC61
:1029100053F0FF0E58EC35F0EEEC52F0FF0E58EC91
:1029200035F02EEC54F0FF0E58EC35F09EEC53F0E1
:10293000FF0E58EC35F01EEC54F0FF0E58EC35F05D
:102940009EEC54F09EEC53F0FF0E58EC35F01DEC6D
:1029500035F0400E26EC35F0BF0E3FEC35F0CEECF6
:1029600053F0FF0E58EC35F0EEEC52F0FF0E58EC41
:1029700035F01EEC53F0FF0E58EC35F049EC39F011
:1029800080B8D6EF14F0070E585CD8B4CBEF14F033
:10299000582AD8EF14F0586A3EB8D8EF14F0010E58
:1029A000436E42EC36F03E88D8EF14F03E98586AF9
:1029B00042EF01F01AEC35F0460E26EC35F0B90E78
:1029C0003FEC35F0000E465CD8B416EF15F0010E62
:1029D000465CD8B417EF16F0020E465CD8B470EF20
:1029E00017F0030E465CD8B484EF18F0040E465C72
:1029F000D8B468EF19F0050E465CD8B477EF1AF03A
:102A0000060E465CD8B49EEF1BF0070E465CD8B4A9
:102A100002EF1DF0080E465CD8B4BAEF1DF0090EA7
:102A2000465CD8B472EF1EF02AEF1FF0BBEC48F002
:102A30003FB21DEF15F0050E4A6E3FB480EF15F062
:102A400080B04EEF15F0070E565CD8B42BEF15F0A2
:102A5000562A50EF15F0566A3EB050EF15F0010EB1
:102A60004A5CD8A438EF15F0080E4A6E4BEF15F00B
:102A7000040E4A5CD8A441EF15F0010E4A6E4BEFEC
:102A800015F0080E4A5CD8A44AEF15F0050E4A6E00
:102A90004BEF15F04A063E8050EF15F03E90566A17
:102AA00084B67EEF15F0070E555CD8B45BEF15F0D9
:102AB000552A80EF15F0556A3EBC80EF15F0080EE0
:102AC0004A5CD8A468EF15F0010E4A6E7BEF15F052
:102AD000010E4A5CD8A471EF15F0040E4A6E7BEF2C
:102AE00015F0050E4A5CD8A47AEF15F0080E4A6E70
:102AF0007BEF15F04A2A3E8C80EF15F03E9C556A1C
:102B00001AEC35F0460E26EC35F0BC0E3FEC35F0F5
:102B1000010E4A5CD8B4BAEF15F0040E4A5CD8B482
:102B2000DDEF15F0080E4A5CD8B4FEEF15F0FF0E8D
:102B300058EC35F01EEC54F0FF0E58EC35F0FEEC7E
:102B400053F0FF0E58EC35F02EEC54F0FF0E58EC1D
:102B500035F0BEEC53F0FF0E58EC35F00EEC53F0B0
:102B6000FF0E58EC35F08EEC54F0000E58EC35F0BA
:102B7000FEEF15F0FF0E58EC35F03EEC53F0FF0E73
:102B800058EC35F00EEC54F0FF0E58EC35F04EECEE
:102B900054F0FF0E58EC35F00EEC53F0FF0E58ECED
:102BA00035F09EEC53F0FF0E58EC35F08EEC53F000
:102BB000FF0E58EC35F0FEEF15F0FF0E58EC35F037
:102BC000DEEC53F0FF0E58EC35F01EEC53F0FF0E28
:102BD00058EC35F02EEC54F0FF0E58EC35F0FEECCE
:102BE00053F0FF0E58EC35F08EEC54F0000E58EC1C
:102BF00035F08EEC54F0000E58EC35F03FB605EF92
:102C000016F03F8611504B6E4C6EC5EC3DF01DEC3E
:102C100035F0400E26EC35F0BD0E3FEC35F040505F
:102C200005EC46F04EEC46F03F8241EF20F014EC0C
:102C300049F03FB21EEF16F0070E4A6E3FA44BEC70
:102C40003DF01AEC35F0460E26EC35F0BC0E3FECAC
:102C500035F0000E4A5CD8B479EF16F0010E4A5CEC
:102C6000D8B4A1EF16F0020E4A5CD8B4C9EF16F042
:102C7000030E4A5CD8B4C9EF16F0040E4A5CD8B40F
:102C8000FDEF16F0050E4A5CD8B4FDEF16F0060E07
:102C90004A5CD8B431EF17F0080E4A5CD8B457EF4D
:102CA00017F0FF0E58EC35F00EEC53F0FF0E58EC19
:102CB00035F05EEC53F0FF0E58EC35F00EEC54F0AE
:102CC000FF0E58EC35F08EEC54F0000E58EC35F059
:102CD0008EEC54F0000E58EC35F08EEC54F0000EF3
:102CE00058EC35F08EEC54F0000E58EC35F057EF00
:102CF00017F0FF0E58EC35F00EEC54F0FF0E58ECC8
:102D000035F04EEC54F0FF0E58EC35F00EEC53F06D
:102D1000FF0E58EC35F09EEC53F0FF0E58EC35F0FA
:102D20008EEC53F0FF0E58EC35F08EEC54F0000EA4
:102D300058EC35F08EEC54F0000E58EC35F057EFAF
:102D400017F0FF0E58EC35F0AEEC53F0FF0E58ECD8
:102D500035F02EEC54F0FF0E58EC35F01EEC54F02C
:102D6000FF0E58EC35F02EEC53F0FF0E58EC35F01A
:102D70000EEC54F0FF0E58EC35F0EEEC52F0FF0E76
:102D800058EC35F0CEEC53F0FF0E58EC35F057EF21
:102D900017F0FF0E58EC35F06EEC53F0FF0E58ECC8
:102DA00035F0BEEC53F0FF0E58EC35F01EEC54F04D
:102DB000FF0E58EC35F0020E4A5CD8B4E7EF16F07F
:102DC0000EEC4FF0FF0E58EC35F0ECEF16F01EEC69
:102DD0004FF0FF0E58EC35F08EEC54F0000E58EC2E
:102DE00035F08EEC54F0000E58EC35F08EEC54F0CB
:102DF000000E58EC35F057EF17F0FF0E58EC35F099
:102E00005EEC53F0FF0E58EC35F0CEEC53F0FF0EB5
:102E100058EC35F09EEC53F0FF0E58EC35F01EECFC
:102E200053F0FF0E58EC35F0040E4A5CD8B420EF96
:102E300017F00EEC4FF0FF0E58EC35F025EF17F0C1
:102E40001EEC4FF0FF0E58EC35F08EEC54F0000EF7
:102E500058EC35F08EEC54F0000E58EC35F057EF8E
:102E600017F0FF0E58EC35F0FEEC53F0FF0E58EC67
:102E700035F0AEEC53F0FF0E58EC35F00EEC53F09D
:102E8000FF0E58EC35F08EEC53F0FF0E58EC35F099
:102E90003EEC53F0FF0E58EC35F08EEC54F0000E83
:102EA00058EC35F08EEC54F0000E58EC35F03FB68F
:102EB0005EEF17F03F8612504B6E4C6EC5EC3DF046
:102EC0001DEC35F0400E26EC35F0BD0E3FEC35F034
:102ED000405005EC46F04EEC46F03F8241EF20F0CA
:102EE0006DEC49F03FB277EF17F0070E4A6E3FA442
:102EF0004BEC3DF01AEC35F0460E26EC35F0BC0EEE
:102F00003FEC35F0000E4A5CD8B4F1EF17F0010E3B
:102F10004A5CD8B423EF18F0020E4A5CD8B423EF11
:102F200018F0030E4A5CD8B423EF18F0080E4A5C80
:102F3000D8B46BEF18F0FF0E58EC35F04EEC53F0B0
:102F4000FF0E58EC35F0DEEC53F0FF0E58EC35F088
:102F5000CEEC53F0FF0E58EC35F00EEC4FF0FF0EB8
:102F600058EC35F00EEC54F0FF0E58EC35F02EEC2A
:102F700053F0FF0E58EC35F09EEC53F0FF0E58EC7A
:102F800035F0040E4A5CD8B4D7EF17F0050E4A5C52
:102F9000D8B4DEEF17F0060E4A5CD8B4E5EF17F0B0
:102FA0000EEC4FF0FF0E58EC35F0EAEF17F03EEC68
:102FB0004FF0FF0E58EC35F0EAEF17F02EEC4FF023
:102FC000FF0E58EC35F0EAEF17F01EEC4FF0FF0E55
:102FD00058EC35F08EEC54F0000E58EC35F06BEFF9
:102FE00018F0FF0E58EC35F01EEC53F0FF0E58ECC5
:102FF00035F02EEC53F0FF0E58EC35F01EEC54F08B
:10300000FF0E58EC35F00EEC53F0FF0E58EC35F097
:103010006EEC53F0FF0E58EC35F08EEC54F0000ED1
:1030200058EC35F08EEC54F0000E58EC35F08EEC88
:1030300054F0000E58EC35F08EEC54F0000E58ECC5
:1030400035F06BEF18F0FF0E58EC35F02EEC53F026
:10305000FF0E58EC35F0AEEC53F0FF0E58EC35F0A7
:10306000DEEC53F0FF0E58EC35F05EEC53F0FF0E43
:1030700058EC35F00EEC53F0FF0E58EC35F0BEEC8A
:1030800053F0FF0E58EC35F01EEC54F0FF0E58ECE8
:1030900035F09EEC53F0FF0E58EC35F0010E4A5C13
:1030A000D8B45FEF18F0020E4A5CD8B466EF18F09F
:1030B0000EEC4FF0FF0E58EC35F06BEF18F02EECE5
:1030C0004FF0FF0E58EC35F06BEF18F01EEC4FF0A0
:1030D000FF0E58EC35F03FB672EF18F03F861350F4
:1030E0004B6E4C6EC5EC3DF01DEC35F0400E26EC01
:1030F00035F0BD0E3FEC35F0405005EC46F04EEC9F
:1031000046F03F8241EF20F0C6EC49F03FB28BEF32
:1031100018F0070E4A6E3FA44BEC3DF01AEC35F068
:10312000460E26EC35F0BC0E3FEC35F0000E4A5C46
:10313000D8B400EF19F0010E4A5CD8B400EF19F0D2
:10314000020E4A5CD8B400EF19F0030E4A5CD8B402
:1031500000EF19F0080E4A5CD8B44FEF19F0FF0EDB
:1031600058EC35F04EEC53F0FF0E58EC35F0DEEC39
:1031700053F0FF0E58EC35F0CEEC53F0FF0E58EC48
:1031800035F02EEC4FF0FF0E58EC35F00EEC54F00D
:10319000FF0E58EC35F02EEC53F0FF0E58EC35F0E6
:1031A0009EEC53F0FF0E58EC35F0040E4A5CD8B498
:1031B000EBEF18F0050E4A5CD8B4F2EF18F0060EEB
:1031C0004A5CD8B4F9EF18F00EEC4FF0FF0E58EC53
:1031D00035F04FEF19F03EEC4FF0FF0E58EC35F0A4
:1031E0004FEF19F02EEC4FF0FF0E58EC35F04FEF8B
:1031F00019F01EEC4FF0FF0E58EC35F04FEF19F0C0
:10320000FF0E58EC35F04EEC53F0FF0E58EC35F055
:10321000DEEC53F0FF0E58EC35F0CEEC53F0FF0E21
:1032200058EC35F01EEC4FF0FF0E58EC35F00EEC7C
:1032300054F0FF0E58EC35F02EEC53F0FF0E58EC26
:1032400035F09EEC53F0FF0E58EC35F0000E4A5C62
:10325000D8B43CEF19F0010E4A5CD8B443EF19F032
:10326000020E4A5CD8B44AEF19F00EEC4FF0FF0E94
:1032700058EC35F04FEF19F03EEC4FF0FF0E58ECE4
:1032800035F04FEF19F02EEC4FF0FF0E58EC35F003
:103290004FEF19F01EEC4FF0FF0E58EC35F03FB633
:1032A00056EF19F03F8614504B6E4C6EC5EC3DF056
:1032B0001DEC35F0400E26EC35F0BD0E3FEC35F040
:1032C000405005EC46F04EEC46F03F8241EF20F0D6
:1032D0001FEC4AF03FB26FEF19F0070E4A6E3FA4A1
:1032E0004BEC3DF01AEC35F0460E26EC35F0BC0EFA
:1032F0003FEC35F0000E4A5CD8B4A4EF19F0010E93
:103300004A5CD8B4C7EF19F0020E4A5CD8B4EAEFB1
:1033100019F0030E4A5CD8B4EAEF19F0040E4A5CC7
:10332000D8B4EAEF19F0050E4A5CD8B425EF1AF0CC
:10333000060E4A5CD8B425EF1AF0080E4A5CD8B4E1
:103340005EEF1AF025EF1AF0FF0E58EC35F0FEECA8
:1033500053F0FF0E58EC35F02EEC54F0FF0E58EC05
:1033600035F0BEEC53F0FF0E58EC35F08EEC54F017
:10337000000E58EC35F08EEC54F0000E58EC35F0A1
:103380008EEC54F0000E58EC35F05EEF1AF0FF0EA4
:1033900058EC35F0FEEC53F0FF0E58EC35F05EECD7
:1033A00054F0FF0E58EC35F01EEC53F0FF0E58ECC5
:1033B00035F08EEC54F0000E58EC35F08EEC54F0F5
:1033C000000E58EC35F08EEC54F0000E58EC35F051
:1033D0005EEF1AF0FF0E58EC35F0FEEC53F0FF0EE6
:1033E00058EC35F05EEC54F0FF0E58EC35F00EEC76
:1033F00054F0FF0E58EC35F02EEC53F0FF0E58EC65
:1034000035F09EEC53F0FF0E58EC35F0020E4A5C9E
:10341000D8B417EF1AF0030E4A5CD8B41EEF1AF0B6
:103420000EEC4FF0FF0E58EC35F05EEF1AF02EEC7C
:103430004FF0FF0E58EC35F05EEF1AF01EEC4FF037
:10344000FF0E58EC35F05EEF1AF0FF0E58EC35F039
:103450001EEC54F0FF0E58EC35F05EEC54F0FF0E0D
:1034600058EC35F00EEC54F0FF0E58EC35F02EEC25
:1034700053F0FF0E58EC35F09EEC53F0FF0E58EC75
:1034800035F0050E4A5CD8B452EF1AF0060E4A5CCD
:10349000D8B459EF1AF00EEC4FF0FF0E58EC35F09F
:1034A0005EEF1AF02EEC4FF0FF0E58EC35F05EEFA9
:1034B0001AF01EEC4FF0FF0E58EC35F03FB665EFFA
:1034C0001AF03F8615504B6E4C6EC5EC3DF01DEC6E
:1034D00035F0400E26EC35F0BD0E3FEC35F0405097
:1034E00005EC46F04EEC46F03F8241EF20F078ECE0
:1034F0004AF03FB27EEF1AF0070E4A6E3FA44BEC43
:103500003DF01AEC35F0460E26EC35F0BC0E3FECE3
:1035100035F0080E4A5CD8B485EF1BF0FF0E58EC6E
:1035200035F00EEC54F0FF0E58EC35F0CEEC53F0C5
:10353000FF0E58EC35F0000E4A5CD8B4D9EF1AF003
:10354000010E4A5CD8B4F4EF1AF0020E4A5CD8B40B
:103550000FEF1BF0030E4A5CD8B40FEF1BF0040E04
:103560004A5CD8B436EF1BF0050E4A5CD8B451EF74
:103570001BF0060E4A5CD8B46CEF1BF09EEC53F0C7
:10358000FF0E58EC35F0FEEC53F0FF0E58EC35F022
:10359000DEEC53F0FF0E58EC35F0CEEC53F0FF0E9E
:1035A00058EC35F09EEC53F0FF0E58EC35F085EFFB
:1035B0001BF0AEEC53F0FF0E58EC35F00EEC54F06F
:1035C000FF0E58EC35F08EEC54F0000E58EC35F050
:1035D0008EEC54F0000E58EC35F08EEC54F0000EEA
:1035E00058EC35F085EF1BF00EEC54F0FF0E58EC64
:1035F00035F03EEC53F0FF0E58EC35F08EEC54F005
:10360000000E58EC35F08EEC54F0000E58EC35F00E
:103610008EEC54F0000E58EC35F085EF1BF0FEEC0C
:1036200053F0FF0E58EC35F02EEC53F0FF0E58EC33
:1036300035F00EEC54F0FF0E58EC35F0020E4A5CFB
:10364000D8B42AEF1BF00EEC4FF0FF0E58EC35F01B
:103650002FEF1BF01EEC4FF0FF0E58EC35F08EEC08
:1036600054F0000E58EC35F085EF1BF07EEC53F073
:10367000FF0E58EC35F02EEC54F0FF0E58EC35F000
:103680000EEC54F0FF0E58EC35F01EEC54F0FF0E2B
:1036900058EC35F08EEC54F0000E58EC35F085EF18
:1036A0001BF01EEC53F0FF0E58EC35F02EEC53F0EF
:1036B000FF0E58EC35F09EEC53F0FF0E58EC35F051
:1036C0008EEC54F0000E58EC35F08EEC54F0000EF9
:1036D00058EC35F085EF1BF00EEC54F0FF0E58EC73
:1036E00035F0DEEC53F0FF0E58EC35F0CEEC53F035
:1036F000FF0E58EC35F09EEC53F0FF0E58EC35F011
:103700008EEC54F0000E58EC35F03FB68CEF1BF009
:103710003F8616504B6E4C6EC5EC3DF01DEC35F0FF
:10372000400E26EC35F0BD0E3FEC35F0405005EC78
:1037300046F04EEC46F03F8241EF20F021EC4BF09A
:103740003FB2A5EF1BF0070E4A6E3FA488EC3DF098
:103750001AEC35F0460E26EC35F0BC0E3FEC35F099
:10376000010E4A5CD8B4FBEF1BF0020E4A5CD8B4E1
:1037700023EF1CF0030E4A5CD8B44BEF1CF0040E90
:103780004A5CD8B473EF1CF0050E4A5CD8B49BEFCA
:103790001CF0060E4A5CD8B4C3EF1CF0080E4A5C5D
:1037A000D8B4E9EF1CF0FF0E58EC35F0DEEC53F026
:1037B000FF0E58EC35F0EEEC52F0FF0E58EC35F001
:1037C000FEEC53F0FF0E58EC35F0AEEC53F0FF0E6C
:1037D00058EC35F08EEC54F0000E58EC35F08EECD1
:1037E00054F0000E58EC35F08EEC54F0000E58EC0E
:1037F00035F0E9EF1CF0FF0E58EC35F0EEEC53F02D
:10380000FF0E58EC35F00EEC53F0FF0E58EC35F08F
:10381000FEEC53F0FF0E58EC35F00EEC53F0FF0EBB
:1038200058EC35F0AEEC53F0FF0E58EC35F08EEC62
:1038300054F0000E58EC35F08EEC54F0000E58ECBD
:1038400035F0E9EF1CF0FF0E58EC35F00EEC53F0BC
:10385000FF0E58EC35F00EEC53F0FF0E58EC35F03F
:10386000FEEC53F0FF0E58EC35F00EEC53F0FF0E6B
:1038700058EC35F0AEEC53F0FF0E58EC35F08EEC12
:1038800054F0000E58EC35F08EEC54F0000E58EC6D
:1038900035F0E9EF1CF0FF0E58EC35F02EEC54F04B
:1038A000FF0E58EC35F0BEEC53F0FF0E58EC35F03F
:1038B0009EEC53F0FF0E58EC35F0CEEC53F0FF0EBB
:1038C00058EC35F00EEC53F0FF0E58EC35F08EEC62
:1038D00053F0FF0E58EC35F0AEEC53F0FF0E58EC01
:1038E00035F0E9EF1CF0FF0E58EC35F03EEC54F0EB
:1038F000FF0E58EC35F0AEEC53F0FF0E58EC35F0FF
:103900008EEC54F0000E58EC35F08EEC54F0000EB6
:1039100058EC35F08EEC54F0000E58EC35F08EEC8F
:1039200054F0000E58EC35F08EEC54F0000E58ECCC
:1039300035F0E9EF1CF0FF0E58EC35F00EEC53F0CB
:10394000FF0E58EC35F0CEEC53F0FF0E58EC35F08E
:10395000AEEC53F0FF0E58EC35F03EEC53F0FF0E9A
:1039600058EC35F0AEEC53F0FF0E58EC35F08EEC21
:1039700054F0000E58EC35F08EEC54F0000E58EC7C
:1039800035F0E9EF1CF0FF0E58EC35F0FEEC52F08C
:10399000FF0E58EC35F06EEC53F0FF0E58EC35F09E
:1039A000DEEC53F0FF0E58EC35F0AEEC53F0FF0EAA
:1039B00058EC35F08EEC54F0000E58EC35F08EECEF
:1039C00054F0000E58EC35F08EEC54F0000E58EC2C
:1039D00035F03FB6F0EF1CF03F8617504B6E4C6E43
:1039E000C5EC3DF01DEC35F0400E26EC35F0BD0E7B
:1039F0003FEC35F0405005EC46F04EEC46F03F828F
:103A000041EF20F0AFEC4BF03FB209EF1DF0070E95
:103A10004A6E3FA488EC3DF01AEC35F0460E26ECD9
:103A200035F0BC0E3FEC35F0010E4A5CD8B44AEFDD
:103A30001DF0020E4A5CD8B458EF1DF0030E4A5C2C
:103A4000D8B461EF1DF0040E4A5CD8B46FEF1DF0DE
:103A5000050E4A5CD8B482EF1DF0060E4A5CD8B45D
:103A600090EF1DF0080E4A5CD8B4A1EF1DF0BBEC3E
:103A70004DF0AEEC53F0FF0E58EC35F08EEC54F0F8
:103A8000000E58EC35F08EEC54F0000E58EC35F08A
:103A9000A1EF1DF030EC4DF0AEEC53F0FF0E58EC02
:103AA00035F08EEC54F0000E58EC35F0A1EF1DF01F
:103AB00048EC4DF0AEEC53F0FF0E58EC35F0A1EFB2
:103AC0001DF065EC4DF0AEEC53F0FF0E58EC35F008
:103AD0008EEC54F0000E58EC35F0A1EF1DF07DECAB
:103AE0004DF0AEEC53F0FF0E58EC35F08EEC54F088
:103AF000000E58EC35F08EEC54F0000E58EC35F01A
:103B0000A1EF1DF090EC4DF0AEEC53F0FF0E58EC31
:103B100035F08EEC54F0000E58EC35F0A1EF1DF0AE
:103B2000A8EC4DF0AEEC53F0FF0E58EC35F08EECF7
:103B300054F0000E58EC35F08EEC54F0000E58ECBA
:103B400035F03FB6A8EF1DF03F8618504B6E4C6E17
:103B5000C5EC3DF01DEC35F0400E26EC35F0BD0E09
:103B60003FEC35F0405005EC46F04EEC46F03F821D
:103B700041EF20F01EEC4CF03FB2C1EF1DF0070EFC
:103B80004A6E3FA488EC3DF01AEC35F0460E26EC68
:103B900035F0BC0E3FEC35F0010E4A5CD8B402EFB4
:103BA0001EF0020E4A5CD8B410EF1EF0030E4A5C01
:103BB000D8B419EF1EF0040E4A5CD8B427EF1EF0FB
:103BC000050E4A5CD8B43AEF1EF0060E4A5CD8B433
:103BD00048EF1EF0080E4A5CD8B459EF1EF0BBEC5B
:103BE0004DF01EEC4FF0FF0E58EC35F08EEC54F01B
:103BF000000E58EC35F08EEC54F0000E58EC35F019
:103C000059EF1EF030EC4DF01EEC4FF0FF0E58EC6B
:103C100035F08EEC54F0000E58EC35F059EF1EF0F4
:103C200048EC4DF01EEC4FF0FF0E58EC35F059EF1C
:103C30001EF065EC4DF01EEC4FF0FF0E58EC35F029
:103C40008EEC54F0000E58EC35F059EF1EF07DEC80
:103C50004DF01EEC4FF0FF0E58EC35F08EEC54F0AA
:103C6000000E58EC35F08EEC54F0000E58EC35F0A8
:103C700059EF1EF090EC4DF01EEC4FF0FF0E58EC9B
:103C800035F08EEC54F0000E58EC35F059EF1EF084
:103C9000A8EC4DF01EEC4FF0FF0E58EC35F08EEC1A
:103CA00054F0000E58EC35F08EEC54F0000E58EC49
:103CB00035F03FB660EF1EF03F8619504B6E4C6EEC
:103CC000C5EC3DF01DEC35F0400E26EC35F0BD0E98
:103CD0003FEC35F0405005EC46F04EEC46F03F82AC
:103CE00041EF20F0A7EC4CF03FB279EF1EF0070E49
:103CF0004A6E3FA488EC3DF01AEC35F0460E26ECF7
:103D000035F0BC0E3FEC35F0010E4A5CD8B4BAEF8A
:103D10001EF0020E4A5CD8B4C8EF1EF0030E4A5CD7
:103D2000D8B4D1EF1EF0040E4A5CD8B4DFEF1EF019
:103D3000050E4A5CD8B4F2EF1EF0060E4A5CD8B409
:103D400000EF1FF0080E4A5CD8B411EF1FF0BBEC77
:103D50004DF00EEC4FF0FF0E58EC35F08EEC54F0B9
:103D6000000E58EC35F08EEC54F0000E58EC35F0A7
:103D700011EF1FF030EC4DF00EEC4FF0FF0E58EC51
:103D800035F08EEC54F0000E58EC35F011EF1FF0CA
:103D900048EC4DF00EEC4FF0FF0E58EC35F011EF03
:103DA0001FF065EC4DF00EEC4FF0FF0E58EC35F0C7
:103DB0008EEC54F0000E58EC35F011EF1FF07DEC56
:103DC0004DF00EEC4FF0FF0E58EC35F08EEC54F049
:103DD000000E58EC35F08EEC54F0000E58EC35F037
:103DE00011EF1FF090EC4DF00EEC4FF0FF0E58EC81
:103DF00035F08EEC54F0000E58EC35F011EF1FF05A
:103E0000A8EC4DF00EEC4FF0FF0E58EC35F08EECB8
:103E100054F0000E58EC35F08EEC54F0000E58ECD7
:103E200035F03FB618EF1FF03F861A504B6E4C6EC0
:103E3000C5EC3DF01DEC35F0400E26EC35F0BD0E26
:103E40003FEC35F0405005EC46F04EEC46F03F823A
:103E500041EF20F07EEC51F0000E58EC35F08EEC86
:103E600051F0000E58EC35F09EEC51F0000E58EC7D
:103E700035F04EEC51F0000E58EC35F08EEC52F06F
:103E8000000E58EC35F0FEEC51F0000E58EC35F019
:103E90007EEC52F0000E58EC35F08EEC54F0FEEC57
:103EA00051F0000E58EC35F02EEC52F01DEC35F0D0
:103EB000400E26EC35F0B90E3FEC35F0000E58EC14
:103EC00035F04EEC51F0000E58EC35F07EEC51F030
:103ED000000E58EC35F01AEC35F0670E26EC35F094
:103EE000BC0E3FEC35F03FB08AEF1FF0000E58ECEF
:103EF00035F0CEEC52F0000E58EC35F08EEC51F06F
:103F0000000E58EC35F06EEC52F0000E58EC35F027
:103F10009CEF1FF0FF0E58EC35F06EEC54F0FF0EE6
:103F200058EC35F02EEC53F0FF0E58EC35F00EEC5B
:103F300054F0FF0E58EC35F01DEC35F0440E26EC35
:103F400035F0BC0E3FEC35F03FB0BBEF1FF0FF0E7D
:103F500058EC35F0BEEC53F0FF0E58EC35F09EEC0B
:103F600054F0FF0E58EC35F0CEEC53F0FF0E58EC49
:103F700035F0CDEF1FF0000E58EC35F01EEC52F08E
:103F8000000E58EC35F08EEC54F0000E58EC35F085
:103F90002EEC52F0000E58EC35F080B0E6EF1FF03A
:103FA000070E565CD8B4D8EF1FF0562AE8EF1FF082
:103FB000566A3EB0E8EF1FF03FB0E2EF1FF03F80DF
:103FC000E3EF1FF03F903E80E8EF1FF03E90566A0F
:103FD00084B601EF20F0070E555CD8B4F3EF1FF064
:103FE000552A03EF20F0556A3EBC03EF20F03FB0A6
:103FF000FDEF1FF03F80FEEF1FF03F903E8C03EF80
:1040000020F03E9C556A80B83FEF20F0070E585CC8
:10401000D8B40EEF20F0582A41EF20F0586A3EB88D
:1040200041EF20F0436A466A42EC36F03FA03BEF96
:1040300020F0080E116E040E126E4B0E136EBB0EA6
:10404000146E9B0E156E880E166E5D905D825D94EB
:104050005D965E905E825E945E967F0E176E7F0E1A
:10406000186E000E196E000E1A6E4D6A4E6A5F6A67
:10407000606B5FEC36F03F903E8842EF01F03E9877
:10408000586A3FB462EF20F080BA60EF20F0070E6C
:10409000575CD8B44FEF20F0572A62EF20F0576AF0
:1040A0003EBA42EF01F0000E436E3E8A466A42EC91
:1040B00036F03F903F923F964A6A4B6A42EF01F0DA
:1040C0003E9A576A42EF01F01AEC35F0410E26ECA9
:1040D00035F0B80E3FEC35F0700E58EC35F0100EA0
:1040E00058EC35F0100E58EC35F0100E58EC35F059
:1040F000000E58EC35F09EEC51F0000E58EC35F007
:10410000CEEC52F0000E58EC35F08EEC54F0FEEC94
:1041100051F0000E58EC35F0CEEC51F0000E58EC9A
:1041200035F01EEC52F0000E58EC35F0EEEC51F08C
:10413000000E58EC35F08EEC54F06EEC52F0000EA0
:1041400058EC35F08EEC51F0000E58EC35F01DECCB
:1041500035F0400E26EC35F0B80E3FEC35F07EEC35
:1041600052F0000E58EC35F07EEC52F0000E58EC98
:1041700035F0CEEC51F0000E58EC35F01EEC52F05C
:10418000000E58EC35F0AEEC51F0000E58EC35F066
:10419000082A210E085CD8B4D3EF20F0100E58EC9A
:1041A00035F0C8EF20F0086A700E58EC35F03AECA4
:1041B00045F01AEC35F0400E26EC35F0B90E3FEC28
:1041C00035F051BE47EF21F0000E495CD8A447EF0F
:1041D00021F0FF0E58EC35F03EEC53F0FF0E58EC9A
:1041E00035F06EEC54F0FF0E58EC35F09EEC54F0C8
:1041F0009EEC53F0FF0E58EC35F06EEC53F0FF0ED2
:1042000058EC35F0BEEC53F0FF0E58EC35F08EEC68
:1042100053F0FF0E58EC35F09EEC54F04EEC54F099
:10422000FF0E58EC35F0FEEC53F0FF0E58EC35F075
:104230006EEC53F01DEC35F0400E26EC35F0B90E67
:104240003FEC35F0FF0E58EC35F01EEC54F0FF0E4D
:1042500058EC35F02EEC53F0FF0E58EC35F09EEC98
:1042600054F03EEC53F0FF0E58EC35F09EEC53F05A
:10427000FF0E58EC35F0EEEC52F0FF0E58EC35F036
:104280004EEC53F0FF0E58EC35F0A3EF21F0000E8A
:1042900058EC35F09EEC51F0000E58EC35F0CEECB9
:1042A00052F0000E58EC35F08EEC54F0FEEC51F06C
:1042B000000E58EC35F0CEEC51F0000E58EC35F015
:1042C0001EEC52F0000E58EC35F0EEEC51F0000E02
:1042D00058EC35F08EEC54F0AEEC52F0000E58EC89
:1042E00035F05EEC52F0000E58EC35F0CEEC51F0AB
:1042F0001DEC35F0400E26EC35F0B90E3FEC35F0F4
:10430000000E58EC35F07EEC52F0000E58EC35F013
:104310008EEC51F0000E58EC35F08EEC54F09EEC23
:1043200051F0000E58EC35F0FEEC51F0000E58EC58
:1043300035F04EEC51F0000E58EC35F0AEEC51F08B
:10434000000E58EC35F01AEC35F0430E26EC35F043
:10435000BA0E3FEC35F01E0E58EC35F0100E58EC4E
:1043600035F0100E58EC35F0100E58EC35F0100EFC
:1043700058EC35F01AEC35F0400E26EC35F0BB0E5B
:104380003FEC35F051BE3DEF22F0010E495CD8A460
:104390003DEF22F0FF0E58EC35F0EEEC52F0FF0E40
:1043A00058EC35F02EEC54F0FF0E58EC35F01EECC6
:1043B00053F0FF0E58EC35F06EEC53F0FF0E58EC56
:1043C00035F0CEEC53F0FF0E58EC35F09EEC54F087
:1043D0003EEC53F0FF0E58EC35F0CEEC53F0FF0EF0
:1043E00058EC35F0FEEC53F0FF0E58EC35F0AEEC27
:1043F00053F0FF0E58EC35F0870E58EC35F0EB0E0D
:1044000058EC35F0ED0E58EC35F0EB0E58EC35F07D
:104410001DEC35F0400E26EC35F0BB0E3FEC35F0D0
:10442000870E58EC35F0FF0E58EC35F01EEC54F0CA
:10443000FF0E58EC35F09EEC54F00EEC54F0FF0EED
:1044400058EC35F02EEC53F0FF0E58EC35F09EECA6
:1044500053F0FF0E58EC35F02EEC53F0FF0E58ECF5
:1044600035F00EEC53F0FF0E58EC35F01EEC54F026
:10447000FF0E58EC35F0AEEF22F0000E58EC35F0A0
:104480004EEC51F0000E58EC35F08EEC52F0000E70
:1044900058EC35F07EEC51F0000E58EC35F0CEECD7
:1044A00051F0000E58EC35F02EEC52F0000E58ECA6
:1044B00035F08EEC54F09EEC51F0000E58EC35F0D7
:1044C0002EEC52F0000E58EC35F05EEC52F0000E7F
:1044D00058EC35F00EEC52F0000E58EC35F0780E3A
:1044E00058EC35F0140E58EC35F0120E58EC35F04F
:1044F000140E58EC35F01DEC35F0400E26EC35F07E
:10450000BB0E3FEC35F0780E58EC35F0000E58EC51
:1045100035F07EEC52F0000E58EC35F08EEC54F095
:104520006EEC52F0000E58EC35F08EEC51F0000EAF
:1045300058EC35F0FEEC51F0000E58EC35F08EECF6
:1045400051F0000E58EC35F06EEC51F0000E58ECC6
:1045500035F07EEC52F0000E58EC35F01AEC35F0E8
:10456000430E26EC35F0BC0E3FEC35F01E0E58EC39
:1045700035F0100E58EC35F0100E58EC35F0100EEA
:1045800058EC35F0100E58EC35F01AEC35F04A0EB8
:1045900026EC35F0BA0E3FEC35F051BEFBEF22F0C1
:1045A00060A1E7EF22F0000E58EC35F02EEC52F04F
:1045B000000E58EC35F01EEC52F0000E58EC35F0C1
:1045C0008EEC54F0000E58EC35F029EF23F0000E7D
:1045D00058EC35F02EEC52F0000E58EC35F09EEC15
:1045E00051F0000E58EC35F09EEC51F0000E58ECF6
:1045F00035F029EF23F0000E495CD8A4D0EF22F06B
:1046000060A117EF23F0FF0E58EC35F0CEEC53F01D
:10461000FF0E58EC35F0BEEC53F0FF0E58EC35F0C1
:104620008EEC54F0000E58EC35F029EF23F0FF0E1D
:1046300058EC35F0CEEC53F0FF0E58EC35F03EEC74
:1046400053F0FF0E58EC35F03EEC53F0FF0E58ECF3
:1046500035F01AEC35F04A0E26EC35F0BC0E3FEC86
:1046600035F051BE0FEF25F05E500F0B616F000E5D
:10467000615DD8B46BEF23F0010E615DD8B4AEEF8D
:1046800023F0020E615DD8B4BAEF23F0030E615D32
:10469000D8B4C6EF23F0040E615DD8B409EF24F05E
:1046A000050E615DD8B415EF24F0060E615DD8B437
:1046B00021EF24F0070E615DD8B464EF24F0080EFA
:1046C000615DD8B470EF24F0090E615DD8B47CEF61
:1046D00024F0BFEF24F0000E58EC35F07EEC4EF0E5
:1046E000000E58EC35F0CEEC4EF0000E58EC35F0E4
:1046F0005EEC51F0000E58EC35F0000E58EC35F041
:10470000CEEC51F0000E58EC35F07EEC52F08EEC11
:1047100054F05EEC52F0000E58EC35F0D2EC54F050
:10472000000E58EC35F0DEEC51F0000E58EC35F090
:104730001DEC35F0400E26EC35F0BC0E3FEC35F0AC
:104740006EEC52F0000E58EC35F07EEC52F0000E9C
:1047500058EC35F08EEC54F0EDEF26F0000E58ECEE
:1047600035F08EEC4EF0000E58EC35F06EEC4EF05D
:1047700075EF23F0000E58EC35F08EEC4EF0000E85
:1047800058EC35F0AEEC4EF075EF23F0000E58EC1F
:1047900035F07EEC4EF0000E58EC35F0CEEC4EF0DD
:1047A000000E58EC35F05EEC51F0000E58EC35F090
:1047B000000E58EC35F0CEEC51F0000E58EC35F010
:1047C0007EEC52F08EEC54F0CEEC51F0000E58EC32
:1047D00035F0CEEC51F0000E58EC35F06EEC52F0A6
:1047E000000E58EC35F01DEC35F0400E26EC35F09F
:1047F000BC0E3FEC35F08EEC54F0000E58EC35F06A
:104800008EEC54F0000E58EC35F08EEC54F0EDEFD9
:1048100026F0000E58EC35F08EEC4EF0000E58EC01
:1048200035F06EEC4EF0D0EF23F0000E58EC35F082
:104830008EEC4EF0000E58EC35F0AEEC4EF0D0EFB2
:1048400023F0000E58EC35F07EEC4EF0000E58ECE4
:1048500035F0CEEC4EF0000E58EC35F05EEC51F039
:10486000000E58EC35F0000E58EC35F0CEEC51F05F
:10487000000E58EC35F07EEC52F08EEC54F0FEEC6D
:1048800051F0000E58EC35F0D2EC54F0000E58EC1C
:1048900035F0DEEC51F0000E58EC35F01DEC35F043
:1048A000400E26EC35F0BC0E3FEC35F06EEC52F0CD
:1048B000000E58EC35F07EEC52F0000E58EC35F05E
:1048C0008EEC54F0EDEF26F0000E58EC35F08EEC47
:1048D0004EF0000E58EC35F06EEC4EF02BEF24F05D
:1048E000000E58EC35F08EEC4EF0000E58EC35F022
:1048F000AEEC4EF02BEF24F0000E58EC35F04EEC01
:1049000051F0000E58EC35F08EEC51F0000E58ECE2
:1049100035F06EEC52F0000E58EC35F09EEC4EF097
:10492000000E58EC35F08EEC54F07EEC51F0000E99
:1049300058EC35F0CEEC51F0000E58EC35F05EEC52
:1049400052F0000E58EC35F08EEC51F0000E58ECA1
:1049500035F01DEC35F0400E26EC35F0BC0E3FEC8A
:1049600035F06EEC51F0000E58EC35F07EEC52F064
:10497000000E58EC35F08EEC54F0EDEF26F0000E02
:1049800058EC35F02EEC52F0000E58EC35F08EEC71
:1049900052F0000E58EC35F07EEC52F0000E58EC60
:1049A00035F08EEC54F02EEC52F0000E58EC35F051
:1049B0009EEC51F0000E58EC35F08EEC54F05EECAD
:1049C00052F0000E58EC35F04EEC51F0000E58EC61
:1049D00035F07E0E58EC35F01DEC35F0400E26EC2F
:1049E00035F0BC0E3FEC35F0040E58EC35F0180EE7
:1049F00058EC35F0200E58EC35F07E0E58EC35F0C2
:104A0000000E58EC35F0AEEC51F0000E58EC35F0DD
:104A10008EEC51F0000E58EC35F0EDEF26F0010E63
:104A2000495CD8A434EF23F05E500F0B616F000E89
:104A3000615DD8B44BEF25F0010E615DD8B48EEF07
:104A400025F0020E615DD8B49AEF25F0030E615D8A
:104A5000D8B4A6EF25F0040E615DD8B4E9EF25F0D7
:104A6000050E615DD8B4F5EF25F0060E615DD8B492
:104A700001EF26F0070E615DD8B444EF26F0080E72
:104A8000615DD8B450EF26F0090E615DD8B45CEFDB
:104A900026F09FEF26F0FF0E58EC35F01EEC4FF09D
:104AA000FF0E58EC35F06EEC4FF0FF0E58EC35F081
:104AB000FEEC52F0FF0E58EC35F0FF0E58EC35F0DE
:104AC0006EEC53F0FF0E58EC35F01EEC54F09EECFB
:104AD00054F0FEEC53F0FF0E58EC35F0E2EC54F0DD
:104AE000FF0E58EC35F07EEC53F0FF0E58EC35F02D
:104AF0001DEC35F0400E26EC35F0BC0E3FEC35F0E9
:104B00000EEC54F0FF0E58EC35F01EEC54F0FF0E96
:104B100058EC35F08EEC54F0EDEF26F0FF0E58EC2B
:104B200035F02EEC4FF0FF0E58EC35F00EEC4FF058
:104B300055EF25F0FF0E58EC35F02EEC4FF0FF0E40
:104B400058EC35F04EEC4FF055EF25F0FF0E58ECD9
:104B500035F01EEC4FF0FF0E58EC35F06EEC4FF0D8
:104B6000FF0E58EC35F0FEEC52F0FF0E58EC35F02D
:104B7000FF0E58EC35F06EEC53F0FF0E58EC35F0AC
:104B80001EEC54F09EEC54F06EEC53F0FF0E58EC1B
:104B900035F06EEC53F0FF0E58EC35F00EEC54F09F
:104BA000FF0E58EC35F01DEC35F0400E26EC35F0DC
:104BB000BC0E3FEC35F08EEC54F0000E58EC35F0A6
:104BC0008EEC54F0000E58EC35F08EEC54F0EDEF16
:104BD00026F0FF0E58EC35F02EEC4FF0FF0E58EC9F
:104BE00035F00EEC4FF0B0EF25F0FF0E58EC35F03D
:104BF0002EEC4FF0FF0E58EC35F04EEC4FF0B0EFCE
:104C000025F0FF0E58EC35F01EEC4FF0FF0E58EC7F
:104C100035F06EEC4FF0FF0E58EC35F0FEEC52F034
:104C2000FF0E58EC35F0FF0E58EC35F06EEC53F0FB
:104C3000FF0E58EC35F01EEC54F09EEC54F09EEC58
:104C400053F0FF0E58EC35F0E2EC54F0FF0E58EC48
:104C500035F07EEC53F0FF0E58EC35F01DEC35F0DE
:104C6000400E26EC35F0BC0E3FEC35F00EEC54F067
:104C7000FF0E58EC35F01EEC54F0FF0E58EC35F0FA
:104C80008EEC54F0EDEF26F0FF0E58EC35F02EECE4
:104C90004FF0FF0E58EC35F00EEC4FF00BEF26F016
:104CA000FF0E58EC35F02EEC4FF0FF0E58EC35F0BF
:104CB0004EEC4FF00BEF26F0FF0E58EC35F0EEEC1B
:104CC00052F0FF0E58EC35F02EEC53F0FF0E58EC7E
:104CD00035F00EEC54F0FF0E58EC35F03EEC4FF092
:104CE000FF0E58EC35F09EEC54F01EEC53F0FF0E26
:104CF00058EC35F06EEC53F0FF0E58EC35F0FEEC4E
:104D000053F0FF0E58EC35F02EEC53F0FF0E58EC3C
:104D100035F01DEC35F0400E26EC35F0BC0E3FECC6
:104D200035F00EEC53F0FF0E58EC35F01EEC54F05D
:104D3000FF0E58EC35F08EEC54F0EDEF26F0FF0E40
:104D400058EC35F0CEEC53F0FF0E58EC35F02EEC6D
:104D500054F0FF0E58EC35F01EEC54F0FF0E58ECFA
:104D600035F09EEC54F0CEEC53F0FF0E58EC35F0DD
:104D70003EEC53F0FF0E58EC35F09EEC54F0FEEC98
:104D800053F0FF0E58EC35F0EEEC52F0FF0E58ECFD
:104D900035F0810E58EC35F01DEC35F0400E26EC68
:104DA00035F0BC0E3FEC35F0FB0E58EC35F0E70E5D
:104DB00058EC35F0DF0E58EC35F0810E58EC35F03C
:104DC000FF0E58EC35F04EEC53F0FF0E58EC35F07A
:104DD0002EEC53F0FF0E58EC35F01AEC35F0400E87
:104DE00026EC35F0BD0E3FEC35F051BE5EEF27F0FE
:104DF000020E495CD8A45EEF27F0FF0E58EC35F0A8
:104E0000FEEC53F0FF0E58EC35F0AEEC53F0FF0E15
:104E100058EC35F00EEC53F0FF0E58EC35F08EECFC
:104E200053F0FF0E58EC35F09EEC54F00EEC54F0BD
:104E3000FF0E58EC35F02EEC53F0FF0E58EC35F029
:104E40009EEC53F0FF0E58EC35F02EEC53F0FF0EB5
:104E500058EC35F00EEC53F0FF0E58EC35F0FD0E2B
:104E600058EC35F0FD0E58EC35F0810E58EC35F06D
:104E7000FD0E58EC35F01DEC35F0400E26EC35F00B
:104E8000BD0E3FEC35F0FD0E58EC35F09EEC54F0C5
:104E9000AEEC53F0FF0E58EC35F0CEEC53F0FF0EB5
:104EA00058EC35F01EEC53F0FF0E58EC35F02EECBC
:104EB00053F0FF0E58EC35F0BDEF27F0000E58EC24
:104EC00035F05EEC52F0000E58EC35F00EEC52F07E
:104ED000000E58EC35F06EEC51F0000E58EC35F049
:104EE000EEEC51F0000E58EC35F08EEC54F06EEC18
:104EF00052F0000E58EC35F08EEC51F0000E58ECEC
:104F000035F0FEEC51F0000E58EC35F08EEC51F01F
:104F1000000E58EC35F06EEC51F0000E58EC35F008
:104F2000020E58EC35F0020E58EC35F07E0E58ECBF
:104F300035F0020E58EC35F01DEC35F0400E26EC45
:104F400035F0BD0E3FEC35F0020E58EC35F08EEC2E
:104F500054F00EEC52F0000E58EC35F02EEC52F0FE
:104F6000000E58EC35F07EEC51F0000E58EC35F0A8
:104F70008EEC51F0000E58EC35F01AEC35F0430E83
:104F800026EC35F0BE0E3FEC35F01E0E58EC35F039
:104F9000100E58EC35F0100E58EC35F0100E58ECA1
:104FA00035F0100E58EC35F01AEC35F04A0E26ECC0
:104FB00035F0BE0E3FEC35F051BE28EF28F060A36F
:104FC00005EF28F0000E58EC35F04EEC51F0000ED5
:104FD00058EC35F08EEC52F0000E58EC35F07EECCB
:104FE00052F0000E58EC35F02EEC52F0000E58EC5A
:104FF00035F08EEC54F0000E58EC35F08EEC54F099
:10500000000E58EC35F074EF28F0000E58EC35F037
:105010000EEC52F0000E58EC35F04EEC51F0000E54
:1050200058EC35F01EEC52F0000E58EC35F08EECDA
:1050300052F0000E58EC35F04EEC51F0000E58ECEA
:1050400035F0FEEC51F0000E58EC35F074EF28F01E
:10505000020E495CD8A4DFEF27F060A353EF28F0DD
:10506000FF0E58EC35F0EEEC52F0FF0E58EC35F038
:105070002EEC54F0FF0E58EC35F01EEC54F0FF0E01
:1050800058EC35F0CEEC53F0FF0E58EC35F08EECCA
:1050900054F0000E58EC35F08EEC54F0000E58EC45
:1050A00035F074EF28F0FF0E58EC35F0AEEC53F00D
:1050B000FF0E58EC35F0EEEC52F0FF0E58EC35F0E8
:1050C000BEEC53F0FF0E58EC35F02EEC54F0FF0E12
:1050D00058EC35F0EEEC52F0FF0E58EC35F09EEC4B
:1050E00053F0FF0E58EC35F080B816EF29F0070E9C
:1050F000585CD8B47FEF28F0582A18EF29F0586A86
:105100003EB818EF29F051AE12EF29F0519E5E50D3
:105110005D6E60515F6E5E500F0B616F000E615DE2
:10512000D8B4BDEF28F0010E615DD8B4C6EF28F009
:10513000020E615DD8B4CFEF28F0030E615DD8B4E4
:10514000D8EF28F0040E615DD8B4E0EF28F0050E2A
:10515000615DD8B4E8EF28F0060E615DD8B4F0EFD9
:1051600028F0070E615DD8B4F8EF28F0080E615DF5
:10517000D8B400EF29F008EF29F016901692169493
:1051800016861698168A168E0EEF29F0169016922D
:10519000169416861688169A168E0EEF29F016901B
:1051A0001692169416861698169A168E0EEF29F0F9
:1051B00016801692168416961698168A0EEF29F007
:1051C00016801692168416961688169A0EEF29F0F7
:1051D00016801692168416961698169A0EEF29F0D7
:1051E00016901692169416961698168A0EEF29F0B7
:1051F00016901692169416961688169A0EEF29F0A7
:1052000016901692169416961698169A0EEF29F086
:1052100016901692169416961688168AFBEC36F09F
:1052200013EF29F0518E3E8818EF29F03E98586A06
:1052300051BE1FEF29F049EC39F038EF29F080BA60
:1052400036EF29F0070E575CD8B42AEF29F0572A19
:1052500038EF29F0576A3EBA38EF29F0519E5D5079
:105260005E6E5F50606F3E8A38EF29F03E9A576A53
:1052700080B08AEF29F0070E565CD8B443EF29F0CE
:10528000562A8CEF29F0566A3EB08CEF29F051BEB9
:1052900055EF29F0020E495CD8B452EF29F0492AA3
:1052A00087EF29F0496A87EF29F0000E495CD8B4EE
:1052B00061EF29F0010E495CD8B46AEF29F080EF64
:1052C00029F060A167EF29F0609187EF29F06081F4
:1052D00087EF29F05E500F0B616F0F0E615DD8B440
:1052E0007AEF29F0090E615DD8B47AEF29F05E2AD1
:1052F00087EF29F05E905E925E945E9687EF29F0CC
:1053000060A386EF29F0609387EF29F060833E80E9
:105310008CEF29F03E90566A84B6DFEF29F0070E35
:10532000555CD8B497EF29F0552AE1EF29F0556A7A
:105330003EBCE1EF29F051BEAAEF29F0000E495C16
:10534000D8B4A6EF29F04906DCEF29F0020E496E29
:10535000DCEF29F0000E495CD8B4B6EF29F0010E5D
:10536000495CD8B4BFEF29F0D5EF29F060A1BCEFBC
:1053700029F06091DCEF29F06081DCEF29F05E50CC
:105380000F0B616F0F0E615DD8B4CFEF29F0000EE7
:10539000615DD8B4CFEF29F05E06DCEF29F05E80C6
:1053A0005E925E945E86DCEF29F060A3DBEF29F06D
:1053B0006093DCEF29F060833E8CE1EF29F03E9CA6
:1053C000556A42EF01F01AEC35F0410E26EC35F04B
:1053D000B80E3FEC35F0700E58EC35F0100E58EC6E
:1053E00035F0100E58EC35F0100E58EC35F0000E7C
:1053F00058EC35F08EEC51F0000E58EC35F08EEC98
:1054000051F0000E58EC35F03EEC52F0000E58EC26
:1054100035F05EEC52F0000E58EC35F02EEC52F008
:10542000000E58EC35F00EEC52F0000E58EC35F052
:105430008EEC54F0AEEC52F0000E58EC35F05EEC11
:1054400052F0000E58EC35F0CEEC51F01DEC35F07A
:10545000400E26EC35F0B80E3FEC35F0000E58EC5F
:1054600035F07EEC52F0000E58EC35F08EEC51F039
:10547000000E58EC35F0082A320E085CD8B446EF1E
:105480002AF0100E58EC35F03BEF2AF0086A700E47
:1054900058EC35F03AEC45F0000E445CD8B458EFC7
:1054A0002AF0010E445CD8B400EF2EF042EF01F078
:1054B0001AEC35F0460E26EC35F0B90E3FEC35F01F
:1054C0006EEC52F0000E58EC35F08EEC51F0000E00
:1054D00058EC35F0FEEC51F0000E58EC35F08EEC47
:1054E00051F0000E58EC35F06EEC51F0000E58EC17
:1054F00035F07EEC52F0000E58EC35F08EEC54F0A6
:105500004EEC51F0000E58EC35F07EEC51F0000EF0
:1055100058EC35F07EEC51F01DEC35F0400E26ECE9
:1055200035F0B90E3FEC35F0000E58EC35F05EEC7E
:1055300052F0000E58EC35F08EEC51F0000E58ECA5
:1055400035F06EEC52F0000E58EC35F06EEC52F087
:10555000000E58EC35F080B0C6EF2AF0070E565C0E
:10556000D8B4B6EF2AF0562AC8EF2AF0566A3EB0F1
:10557000C8EF2AF00B0E475CD8B4C2EF2AF0472AD6
:10558000C3EF2AF0476A3E80C8EF2AF03E90566A81
:1055900084B6E4EF2AF0070E555CD8B4D3EF2AF0B6
:1055A000552AE6EF2AF0556A3EBCE6EF2AF0000ED7
:1055B000475CD8B4DFEF2AF04706E1EF2AF00B0E84
:1055C000476E3E8CE6EF2AF03E9C556A1AEC35F0A9
:1055D0004A0E26EC35F0BB0E3FEC35F0000E475C72
:1055E000D8B407EF2BF0000E58EC35F06EEC4EF00F
:1055F000000E58EC35F06EEC4EF0000E58EC35F025
:10560000BEEC51F0000E58EC35F019EF2BF0FF0E08
:1056100058EC35F00EEC4FF0FF0E58EC35F00EEC78
:105620004FF0FF0E58EC35F05EEC53F0FF0E58ECE7
:1056300035F01AEC35F0670E26EC35F0BB0E3FEC7A
:1056400035F0010E475CD8B43AEF2BF0000E58EC61
:1056500035F06EEC4EF0000E58EC35F07EEC4EF06E
:10566000000E58EC35F0BEEC51F0000E58EC35F061
:105670004CEF2BF0FF0E58EC35F00EEC4FF0FF0E18
:1056800058EC35F01EEC4FF0FF0E58EC35F05EECA8
:1056900053F0FF0E58EC35F01DEC35F0440E26ECBF
:1056A00035F0BB0E3FEC35F0020E475CD8B46DEF21
:1056B0002BF0000E58EC35F06EEC4EF0000E58EC6E
:1056C00035F08EEC4EF0000E58EC35F0BEEC51F09B
:1056D000000E58EC35F07FEF2BF0FF0E58EC35F054
:1056E0000EEC4FF0FF0E58EC35F02EEC4FF0FF0EA5
:1056F00058EC35F05EEC53F0FF0E58EC35F01DEC35
:1057000035F0610E26EC35F0BB0E3FEC35F0030EA4
:10571000475CD8B4A0EF2BF0000E58EC35F06EECDF
:105720004EF0000E58EC35F09EEC4EF0000E58ECAA
:1057300035F0BEEC51F0000E58EC35F0B2EF2BF026
:10574000FF0E58EC35F00EEC4FF0FF0E58EC35F034
:105750003EEC4FF0FF0E58EC35F05EEC53F0FF0ED0
:1057600058EC35F01AEC35F04A0E26EC35F0BC0E4C
:105770003FEC35F0040E475CD8B4D3EF2BF0000EAD
:1057800058EC35F06EEC4EF0000E58EC35F0AEEC07
:105790004EF0000E58EC35F0BEEC51F0000E58EC17
:1057A00035F0E5EF2BF0FF0E58EC35F00EEC4FF036
:1057B000FF0E58EC35F04EEC4FF0FF0E58EC35F084
:1057C0005EEC53F0FF0E58EC35F01AEC35F0670E36
:1057D00026EC35F0BC0E3FEC35F0050E475CD8B436
:1057E00006EF2CF0000E58EC35F06EEC4EF0000E8B
:1057F00058EC35F0BEEC4EF0000E58EC35F0BEEC37
:1058000051F0000E58EC35F018EF2CF0FF0E58EC6C
:1058100035F00EEC4FF0FF0E58EC35F05EEC4FF02B
:10582000FF0E58EC35F05EEC53F0FF0E58EC35F0FF
:105830001DEC35F0440E26EC35F0BC0E3FEC35F097
:10584000060E475CD8B439EF2CF0000E58EC35F05A
:105850006EEC4EF0000E58EC35F0CEEC4EF0000E33
:1058600058EC35F0BEEC51F0000E58EC35F04BEF33
:105870002CF0FF0E58EC35F00EEC4FF0FF0E58EC0C
:1058800035F06EEC4FF0FF0E58EC35F05EEC53F057
:10589000FF0E58EC35F01DEC35F0610E26EC35F0BE
:1058A000B40E3FEC35F0070E475CD8B46CEF2CF02B
:1058B000000E58EC35F06EEC4EF0000E58EC35F062
:1058C000DEEC4EF0000E58EC35F0BEEC51F0000E60
:1058D00058EC35F07EEF2CF0FF0E58EC35F00EEC66
:1058E0004FF0FF0E58EC35F07EEC4FF0FF0E58EC09
:1058F00035F05EEC53F0FF0E58EC35F01AEC35F055
:105900004A0E26EC35F0BD0E3FEC35F0080E475C34
:10591000D8B49FEF2CF0000E58EC35F06EEC4EF042
:10592000000E58EC35F0EEEC4EF0000E58EC35F071
:10593000BEEC51F0000E58EC35F0B1EF2CF0FF0E3C
:1059400058EC35F00EEC4FF0FF0E58EC35F08EECC5
:105950004FF0FF0E58EC35F05EEC53F0FF0E58ECB4
:1059600035F01AEC35F0670E26EC35F0BD0E3FEC45
:1059700035F0090E475CD8B4D2EF2CF0000E58EC8D
:1059800035F06EEC4EF0000E58EC35F0FEEC4EF0BB
:10599000000E58EC35F0BEEC51F0000E58EC35F02E
:1059A000E4EF2CF0FF0E58EC35F00EEC4FF0FF0E4C
:1059B00058EC35F09EEC4FF0FF0E58EC35F05EECF5
:1059C00053F0FF0E58EC35F01AEC35F04A0E26EC89
:1059D00035F0BE0E3FEC35F00A0E475CD8B420EF30
:1059E0002DF0000E58EC35F02EEC52F0000E58EC75
:1059F00035F07EEC52F0000E58EC35F0BEEC51F074
:105A0000000E58EC35F08EEC51F0000E58EC35F0ED
:105A10005EEC52F0000E58EC35F08EEC54F06EEC6B
:105A200052F0000E58EC35F08EEC51F0000E58ECB0
:105A300035F07EEC52F0000E58EC35F04DEF2DF0C5
:105A4000FF0E58EC35F0CEEC53F0FF0E58EC35F06D
:105A50001EEC54F0FF0E58EC35F05EEC53F0FF0EE8
:105A600058EC35F02EEC53F0FF0E58EC35F0FEEC10
:105A700053F0FF0E58EC35F09EEC54F00EEC54F061
:105A8000FF0E58EC35F02EEC53F0FF0E58EC35F0CD
:105A90001EEC54F0FF0E58EC35F01AEC35F04A0EBF
:105AA00026EC35F0BF0E3FEC35F00B0E475CD8B45A
:105AB000A0EF2DF0000E58EC35F04EEC51F0000E3A
:105AC00058EC35F0FEEC51F0000E58EC35F0FEECE1
:105AD00051F0000E58EC35F08EEC54F05EEC52F0C4
:105AE000000E58EC35F08EEC51F0000E58EC35F00D
:105AF000AEEC51F0000E58EC35F0CEEC51F0000E4B
:105B000058EC35F06EEC52F0000E58EC35F01DEC10
:105B100035F0400E26EC35F0BF0E3FEC35F07EEC54
:105B200052F0000E58EC35F08EEC51F0000E58ECAF
:105B300035F05EEC52F0000E58EC35F0E4EF2DF04D
:105B4000FF0E58EC35F0EEEC52F0FF0E58EC35F04D
:105B50009EEC53F0FF0E58EC35F09EEC53F0FF0E28
:105B600058EC35F09EEC54F0FEEC53F0FF0E58EC80
:105B700035F02EEC53F0FF0E58EC35F04EEC53F0B0
:105B8000FF0E58EC35F06EEC53F0FF0E58EC35F08C
:105B90000EEC54F0FF0E58EC35F01DEC35F0400ED5
:105BA00026EC35F0BF0E3FEC35F01EEC54F0FF0E46
:105BB00058EC35F02EEC53F0FF0E58EC35F0FEECBF
:105BC00053F0FF0E58EC35F049EC39F080B8FCEF9B
:105BD0002DF0070E585CD8B4F1EF2DF0582AFEEFE7
:105BE0002DF0586A3EB8FEEF2DF0010E446E42ECE7
:105BF00036F03E88FEEF2DF03E98586A42EF01F0F5
:105C00001AEC35F0460E26EC35F0B90E3FEC35F0C7
:105C1000000E475CD8B441EF2EF0010E475CD8B4BB
:105C200049EF2EF0020E475CD8B451EF2EF0030E70
:105C3000475CD8B459EF2EF0040E475CD8B461EF3E
:105C40002EF0050E475CD8B469EF2EF0060E475CC7
:105C5000D8B471EF2EF0070E475CD8B479EF2EF070
:105C6000080E475CD8B481EF2EF0090E475CD8B41B
:105C700089EF2EF00A0E475CD8B491EF2EF0EBEFCF
:105C80002EF0BBEC48F05DEC40F0F6EC40F07EEF1F
:105C90002FF014EC49F05DEC40F0F6EC40F07EEFB4
:105CA0002FF06DEC49F05DEC40F0F6EC40F07EEF4B
:105CB0002FF0C6EC49F05DEC40F0F6EC40F07EEFE2
:105CC0002FF01FEC4AF05DEC40F0F6EC40F07EEF78
:105CD0002FF078EC4AF05DEC40F0F6EC40F07EEF0F
:105CE0002FF021EC4BF05DEC40F0F6EC40F07EEF55
:105CF0002FF0AFEC4BF05DEC40F0F6EC40F07EEFB7
:105D00002FF01EEC4CF05DEC40F0F6EC40F07EEF36
:105D10002FF0A7EC4CF05DEC40F0F6EC40F07EEF9D
:105D20002FF0000E58EC35F02EEC52F0000E58EC2F
:105D300035F07EEC52F0000E58EC35F0BEEC51F030
:105D4000000E58EC35F08EEC51F0000E58EC35F0AA
:105D50005EEC52F0000E58EC35F08EEC54F06EEC28
:105D600052F0000E58EC35F08EEC51F0000E58EC6D
:105D700035F07EEC52F0000E58EC35F01DEC35F0AD
:105D8000400E26EC35F0B90E3FEC35F0000E58EC25
:105D900035F0000E58EC35F0AEEC52F0000E58EC39
:105DA00035F05EEC52F0000E58EC35F0CEEC51F0D0
:105DB000000E58EC35F07EEC52F0000E58EC35F049
:105DC0008EEC51F0000E58EC35F05DEC40F0F6EC46
:105DD00040F07EEF2FF04EEC51F0000E58EC35F015
:105DE000FEEC51F0000E58EC35F0FEEC51F0000ED8
:105DF00058EC35F08EEC54F05EEC52F0000E58EC9E
:105E000035F08EEC51F0000E58EC35F0AEEC51F060
:105E1000000E58EC35F0CEEC51F0000E58EC35F099
:105E20006EEC52F0000E58EC35F07EEC52F01DECAA
:105E300035F0400E26EC35F0B90E3FEC35F0000E93
:105E400058EC35F08EEC51F0000E58EC35F05EEC6D
:105E500052F0000E58EC35F08EEC54F0AEEC52F0EF
:105E6000000E58EC35F05EEC52F0000E58EC35F0B8
:105E7000CEEC51F0000E58EC35F07EEC52F0000EF6
:105E800058EC35F08EEC51F0000E58EC35F05DEC2E
:105E900040F080B87CEF2FF0070E585CD8B454EF78
:105EA0002FF0582A7EEF2FF0586A3EB87EEF2FF081
:105EB0003FAC75EF2FF042EC36F026EC55F039ECA4
:105EC00055F04CEC55F05FEC55F072EC55F085EC6C
:105ED00055F098EC55F0ABEC55F0BEEC55F0D1EC2C
:105EE00055F0E4EC55F0F8EC55F0446A476A3F9CF5
:105EF0003F903E8842EF01F03E98586A80BA42EFE8
:105F000001F0070E575CD8B489EF2FF0572A42EF03
:105F100001F0576A000E446E3E8A476A42EC36F042
:105F20003F9C42EF01F01AEC35F0410E26EC35F0C3
:105F3000B80E3FEC35F0700E58EC35F0100E58EC02
:105F400035F0100E58EC35F0100E58EC35F0000E10
:105F500058EC35F02EEC52F0000E58EC35F07EEC9B
:105F600052F0000E58EC35F0BEEC51F0000E58EC3B
:105F700035F08EEC51F0000E58EC35F05EEC52F03E
:105F8000000E58EC35F08EEC54F06EEC52F0000E32
:105F900058EC35F08EEC51F0000E58EC35F07EECFC
:105FA00052F0000E58EC35F07EEC52F01DEC35F05E
:105FB000400E26EC35F0B80E3FEC35F0000E58ECF4
:105FC00035F0CEEC51F0000E58EC35F01EEC52F0EE
:105FD000000E58EC35F0AEEC51F0000E58EC35F0F8
:105FE000082A2C0E085CD8B4FBEF2FF0100E58ECEA
:105FF00035F0F0EF2FF0086A700E58EC35F03AECFF
:1060000045F01AEC35F0460E26EC35F0BF0E3FECAD
:1060100035F06EEC52F0000E58EC35F02EEC52F0EC
:10602000000E58EC35F09EEC51F0000E58EC35F0B7
:106030007EEC52F0000E58EC35F0AEEC52F0000E53
:1060400058EC35F04EEC51F0000E58EC35F05EECAB
:1060500052F0000E58EC35F08EEC51F0000E58EC7A
:1060600035F08EEC54F09EEC52F01DEC35F0400E05
:1060700026EC35F0BF0E3FEC35F0000E58EC35F055
:106080008EEC51F0000E58EC35F05EEC52F0000E44
:1060900058EC35F06EEC52F0000E58EC35F0CEECCA
:1060A00051F0000E58EC35F02EEC52F0000E58EC8A
:1060B00035F01EEC52F0000E58EC35F08EEC54F03A
:1060C000000E58EC35F08EEC4EF0000E58EC35F02A
:1060D000000E58EC35F0400E58EC35F0000E58EC40
:1060E00035F06EEC4EF0000E58EC35F06EEC4EF0E4
:1060F000000E58EC35F01AEC35F0400E26EC35F079
:10610000B90E3FEC35F04DBEBFEF30F0000E485CED
:10611000D8A4BFEF30F0FF0E58EC35F02EEC53F062
:10612000FF0E58EC35F0FEEC53F0FF0E58EC35F056
:10613000FEEC53F0FF0E58EC35F0CEEC53F0FF0EB2
:1061400058EC35F0FEEC53F0FF0E58EC35F09EECB9
:1061500054F05EEC53F0FF0E58EC35F0CEEC53F0FB
:10616000FF0E58EC35F09EEC53F0FF0E58EC35F076
:106170001EEC53F0FF0E58EC35F0F1EF30F0000E4E
:1061800058EC35F08EEC51F0000E58EC35F05EEC2A
:1061900052F0000E58EC35F05EEC52F0000E58EC68
:1061A00035F02EEC52F0000E58EC35F05EEC52F06B
:1061B000000E58EC35F08EEC54F0BEEC51F0000EB1
:1061C00058EC35F02EEC52F0000E58EC35F0FEECA9
:1061D00051F0000E58EC35F07EEC51F0000E58EC0A
:1061E00035F01AEC35F0430E26EC35F0BA0E3FECE4
:1061F00035F01E0E58EC35F0100E58EC35F0100E40
:1062000058EC35F0100E58EC35F0100E58EC35F017
:106210001AEC35F0400E26EC35F0BB0E3FEC35F0B5
:106220004DBE47EF31F0010E485CD8A447EF31F086
:10623000FF0E58EC35F01EEC54F0FF0E58EC35F024
:106240005EEC54F0FF0E58EC35F09EEC54F0CEECC2
:1062500053F0FF0E58EC35F02EEC54F0FF0E58ECD6
:1062600035F01EEC54F0FF0E58EC35F0DEEC53F038
:10627000FF0E58EC35F02EEC54F0FF0E58EC35F0D4
:106280001EEC54F0FF0E58EC35F074EF31F0000EB8
:1062900058EC35F07EEC52F0000E58EC35F0BEECC8
:1062A00052F0000E58EC35F08EEC54F02EEC52F01B
:1062B000000E58EC35F08EEC52F0000E58EC35F034
:1062C0007EEC52F0000E58EC35F03EEC52F0000E31
:1062D00058EC35F08EEC52F0000E58EC35F07EECB8
:1062E00052F0000E58EC35F01AEC35F0430E26EC67
:1062F00035F0BC0E3FEC35F01E0E58EC35F0100EAC
:1063000058EC35F0100E58EC35F0100E58EC35F016
:10631000100E58EC35F01AEC35F0400E26EC35F046
:10632000BD0E3FEC35F04DBECFEF31F0020E485CB4
:10633000D8A4CFEF31F0FF0E58EC35F00EEC54F04E
:10634000FF0E58EC35F02EEC53F0FF0E58EC35F004
:106350009EEC53F0FF0E58EC35F02EEC53F0FF0E90
:1063600058EC35F00EEC53F0FF0E58EC35F01EEC07
:1063700054F0FF0E58EC35F09EEC54F02EEC54F037
:10638000FF0E58EC35F00EEC54F0FF0E58EC35F0E3
:10639000FEEC52F0FF0E58EC35F001EF32F0000E3B
:1063A00058EC35F06EEC52F0000E58EC35F08EECF7
:1063B00051F0000E58EC35F0FEEC51F0000E58ECA8
:1063C00035F08EEC51F0000E58EC35F06EEC51F0DB
:1063D000000E58EC35F07EEC52F0000E58EC35F023
:1063E0008EEC54F08EEC52F0000E58EC35F06EEC62
:1063F00052F0000E58EC35F05EEC51F0000E58EC07
:1064000035F01AEC35F0430E26EC35F0BE0E3FECBD
:1064100035F01E0E58EC35F0100E58EC35F0100E1D
:1064200058EC35F0100E58EC35F0100E58EC35F0F5
:106430004DBE56EF32F080B036EF32F0070E565CAC
:10644000D8B426EF32F0562A38EF32F0566A3EB012
:1064500038EF32F0020E485CD8B432EF32F0482AFE
:1064600033EF32F0486A3E8038EF32F03E90566AA1
:1064700084B654EF32F0070E555CD8B443EF32F0D7
:10648000552A56EF32F0556A3EBC56EF32F0000EF8
:10649000485CD8B44FEF32F0480651EF32F0020EAC
:1064A000486E3E8C56EF32F03E9C556A4DBE70EF02
:1064B00032F080B86EEF32F0070E585CD8B464EF5B
:1064C00032F0582A70EF32F0586A3EB870EF32F06E
:1064D0004D8E4D504E6E3E8870EF32F03E98586AA9
:1064E0004DAE8AEF32F080BA88EF32F0070E575C7B
:1064F000D8B47EEF32F0572A8AEF32F0576A3EBAAC
:106500008AEF32F04D9E4D504E6E3E8A8AEF32F049
:106510003E9A576A4DAEA6EF32F080B8A4EF32F043
:10652000070E585CD8B498EF32F0582AA6EF32F034
:10653000586A3EB8A6EF32F04E504D6E4D9E42EC7A
:1065400036F03E88A6EF32F03E98586A4DAE01EF25
:1065500033F080B0D3EF32F0070E565CD8B4B4EF0E
:1065600032F0562AD5EF32F0566A3EB0D5EF32F00F
:10657000000E485CD8B4C9EF32F0010E485CD8B4C4
:10658000CCEF32F0020E485CD8B4CFEF32F0D0EF4F
:1065900032F04E70D0EF32F04E72D0EF32F04E74D7
:1065A0003E80D5EF32F03E90566A84B6FFEF32F06F
:1065B000070E555CD8B4E0EF32F0552A01EF33F006
:1065C000556A3EBC01EF33F0000E485CD8B4F5EFDD
:1065D00032F0010E485CD8B4F8EF32F0020E485C9D
:1065E000D8B4FBEF32F0FCEF32F04E70FCEF32F03B
:1065F0004E72FCEF32F04E743E8C01EF33F03E9C55
:10660000556A1AEC35F04A0E26EC35F0BA0E3FEC1E
:1066100035F0000E485CD8A446EF33F04DAE46EF9F
:1066200033F04EA02DEF33F0FF0E58EC35F05EEC5A
:1066300053F0FF0E58EC35F0CEEC53F0FF0E58EC53
:1066400035F09EEC53F0FF0E58EC35F01EEC53F095
:10665000FF0E58EC35F079EF33F0FF0E58EC35F0C3
:106660003EEC53F0FF0E58EC35F0FEEC53F0FF0E0D
:1066700058EC35F02EEC53F0FF0E58EC35F02EECC4
:1066800053F0FF0E58EC35F079EF33F04EA062EF87
:1066900033F0000E58EC35F0BEEC51F0000E58EC23
:1066A00035F02EEC52F0000E58EC35F0FEEC51F0C7
:1066B000000E58EC35F07EEC51F0000E58EC35F041
:1066C00079EF33F0000E58EC35F09EEC51F0000EEF
:1066D00058EC35F05EEC52F0000E58EC35F08EECD4
:1066E00051F0000E58EC35F08EEC51F0000E58ECE5
:1066F00035F01AEC35F04A0E26EC35F0BC0E3FECC6
:1067000035F0010E485CD8A400EF34F04DAE00EF38
:1067100034F04EA2C6EF33F0FF0E58EC35F06EECBD
:1067200053F0FF0E58EC35F0BEEC53F0FF0E58EC72
:1067300035F01EEC54F0FF0E58EC35F02EEC53F013
:10674000FF0E58EC35F0FEEC53F0FF0E58EC35F030
:106750009EEC53F0FF0E58EC35F0CEEC53F0FF0EEC
:1067600058EC35F00EEC53F0FF0E58EC35F08EEC93
:1067700053F01DEC35F0400E26EC35F0BC0E3FEC2E
:1067800035F0FF0E58EC35F075EF34F0FF0E58EC95
:1067900035F03EEC53F0FF0E58EC35F0FEEC53F0C4
:1067A000FF0E58EC35F02EEC53F0FF0E58EC35F0A0
:1067B0002EEC53F0FF0E58EC35F08EEC54F0000E3A
:1067C00058EC35F08EEC54F0000E58EC35F08EECB1
:1067D00054F0000E58EC35F08EEC54F0000E58ECEE
:1067E00035F08EEC54F01DEC35F0400E26EC35F013
:1067F000BC0E3FEC35F0000E58EC35F075EF34F080
:106800004EA23DEF34F0000E58EC35F0CEEC51F0D6
:10681000000E58EC35F01EEC52F0000E58EC35F03E
:106820007EEC52F0000E58EC35F08EEC51F0000E7C
:1068300058EC35F05EEC52F0000E58EC35F0FEEC02
:1068400051F0000E58EC35F02EEC52F0000E58ECE2
:1068500035F06EEC51F0000E58EC35F0EEEC51F0E6
:106860001DEC35F0400E26EC35F0BC0E3FEC35F05B
:10687000000E58EC35F075EF34F0000E58EC35F0A2
:106880009EEC51F0000E58EC35F05EEC52F0000E2C
:1068900058EC35F08EEC51F0000E58EC35F08EECE3
:1068A00051F0000E58EC35F08EEC54F0000E58EC20
:1068B00035F08EEC54F0000E58EC35F08EEC54F0C0
:1068C000000E58EC35F08EEC54F0000E58EC35F01C
:1068D0008EEC54F01DEC35F0400E26EC35F0BC0E7D
:1068E0003FEC35F0000E58EC35F01AEC35F04A0E5E
:1068F00026EC35F0BE0E3FEC35F0020E485CD8A415
:10690000CEEF34F04DAECEEF34F04EA4ABEF34F01A
:10691000FF0E58EC35F0EEEC52F0FF0E58EC35F06F
:106920002EEC54F0FF0E58EC35F01EEC54F0FF0E38
:1069300058EC35F0CEEC53F0FF0E58EC35F08EEC01
:1069400054F0000E58EC35F08EEC54F0000E58EC7C
:1069500035F015EF35F0FF0E58EC35F0AEEC53F096
:10696000FF0E58EC35F0EEEC52F0FF0E58EC35F01F
:10697000BEEC53F0FF0E58EC35F02EEC54F0FF0E49
:1069800058EC35F0EEEC52F0FF0E58EC35F09EEC82
:1069900053F0FF0E58EC35F015EF35F04EA4F4EF40
:1069A00034F0000E58EC35F04EEC51F0000E58EC7F
:1069B00035F08EEC52F0000E58EC35F07EEC52F0D3
:1069C000000E58EC35F02EEC52F0000E58EC35F07D
:1069D0008EEC54F0000E58EC35F08EEC54F0000EB6
:1069E00058EC35F015EF35F0000E58EC35F00EECA4
:1069F00052F0000E58EC35F04EEC51F0000E58EC11
:106A000035F01EEC52F0000E58EC35F08EEC52F0E2
:106A1000000E58EC35F04EEC51F0000E58EC35F00D
:106A2000FEEC51F0000E58EC35F04DAE49EC39F06B
:106A300042EF01F08C888B9E12008C988B8E120096
:106A40008C888B8E12008C988B9E1200016E1FEC2E
:106A500036F001508A6E8C9C8C9E000000008C8A5F
:106A60000000000000000000000000000000000026
:106A70008C9A000000000000000000001200026E6E
:106A80001FEC36F002508A6E8C9C8C9E0000000039
:106A90008C8A0000000000000000000000000000E0
:106AA00000008C9A000000000000000000001200AE
:106AB000006E1FEC36F03FBE74EC35F000508A6E6D
:106AC0008C9C8C8E000000008C8A0000000000006E
:106AD000000000000000000000008C9A0000000090
:106AE0000000000000001200000E525CD8B499EFC4
:106AF00035F0010E525CD8B4B2EF35F0020E525CA4
:106B0000D8B4C9EF35F0030E525CD8B4DEEF35F0DF
:106B1000040E525CD8B4F1EF35F0050E525CD8B4D7
:106B200002EF36F0060E525CD8B411EF36F01EEFCD
:106B300036F051B0A7EF35F000420042004200426B
:106B4000004200420042010E00161EEF36F00046E1
:106B5000004600460046004600460046800E0016ED
:106B60001EEF36F051B0BFEF35F000420042004258
:106B7000004200420042030E00161EEF36F00046AF
:106B800000460046004600460046C00E00161EEFB6
:106B900036F051B0D5EF35F00042004200420042DD
:106BA0000042070E00161EEF36F000460046004673
:106BB00000460046E00E00161EEF36F051B0E9EF39
:106BC00035F000420042004200420F0E00161EEF58
:106BD00036F00046004600460046F00E00161EEF56
:106BE00036F051B0FBEF35F00042004200421F0E7C
:106BF00000161EEF36F0004600460046F80E00165E
:106C00001EEF36F051B00BEF36F0004200423F0E5F
:106C100000161EEF36F000460046FC0E00161EEF72
:106C200036F051B019EF36F000427F0E00161EEF1D
:106C300036F00046FE0E00161EEF36F012000F0171
:106C4000FF0E936E00018C8C8C9E000000008C8ADD
:106C50000000000000000000000000000000000034
:106C60008C9A0000000000000000000000000000FE
:106C7000000081BE27EF36F08C9C0F01000E936E52
:106C80000001120020EC35F0400E26EC35F0B80E75
:106C90003FEC35F0000E58EC35F0012A800E015C17
:106CA000D8A44AEF36F0022A40EC35F0400E26EC2C
:106CB00035F0C00E025CD8A44AEF36F012008B808B
:106CC00000008B92ACEC42F08B82ACEC42F07CEC9E
:106CD00036F092EC36F0BCEC36F0D1EC36F0E6EC67
:106CE00036F0FBEC36F010EC37F025EC37F03AECF0
:106CF00037F04FEC37F012008B90000064EC37F067
:106D00008B9400008B8600008B960000000E386E7E
:106D10008FEC37F011503C6EA4EC37F08B948B96CF
:106D20008B8012008B9064EC37F08B9400008B8684
:106D300000008B960000010E386E8FEC37F0125079
:106D40003C6EA4EC37F08B948B968B8012008B906A
:106D500064EC37F08B9400008B8600008B9600006B
:106D6000010E386E8FEC37F0400E3C6EA4EC37F01D
:106D70008B948B968B8012008B9064EC37F08B9405
:106D800000008B8600008B960000020E386E8FECA0
:106D900037F013503C6EA4EC37F08B948B968B80BD
:106DA00012008B9064EC37F08B9400008B8600000F
:106DB0008B960000030E386E8FEC37F014503C6E4B
:106DC000A4EC37F08B948B968B8012008B9064EC44
:106DD00037F08B9400008B8600008B960000040E29
:106DE000386E8FEC37F015503C6EA4EC37F08B9476
:106DF0008B968B8012008B9064EC37F08B940000A4
:106E00008B8600008B960000050E386E8FEC37F0F5
:106E100016503C6EA4EC37F08B948B968B8012004E
:106E20008B9064EC37F08B9400008B8600008B967F
:106E30000000060E386E8FEC37F017503C6EA4EC55
:106E400037F08B948B968B8012008B9064EC37F02C
:106E50008B9400008B8600008B960000070E386E26
:106E60008FEC37F018503C6EA4EC37F08B948B9677
:106E70008B8012008B9064EC37F08B9400008B8633
:106E800000008B960000080E386E8FEC37F019501A
:106E90003C6EA4EC37F08B948B968B8012008B9019
:106EA00064EC37F08B9400008B8600008B9600001A
:106EB000090E386E8FEC37F01A503C6EA4EC37F0A8
:106EC0008B948B968B8012008B9400008B86000035
:106ED0008B9600008B9400008B8600008B96000040
:106EE0008B8400008B8600008B9600008B94000042
:106EF0008B8600008B9600008B9400008B86000030
:106F00008B9600008B9400008B8600008B9600000F
:106F10008B9400008B8600008B960000120038BE18
:106F200095EF37F08B9497EF37F08B8400008B86CA
:106F300000008B960000392A3846080E395CD8A428
:106F40008FEF37F0396A12003CBEAAEF37F08B940E
:106F5000ACEF37F08B8400008B8600008B9600002E
:106F60003A2A3C46080E3A5CD8A4A4EF37F03A6AB5
:106F700012008B9064EC37F08B9400008B8600003D
:106F80008B9600000A0E386E8FEC37F08B80000075
:106F9000000000008B9064EC37F08B8400008B863F
:106FA00000008B960000000000000000DCEC37F0D1
:106FB0008B948B968B8012008B8683A0E3EF37F047
:106FC0003B80E4EF37F03B903A2A8B96080E3A5C10
:106FD000D8B4EEEF37F03B46DCEF37F03A6A3D2AA3
:106FE000010E3D5CD8A4F9EF37F03B501B6EDCEF8F
:106FF00037F0020E3D5CD8A402EF38F03B501C6E17
:10700000DCEF37F0030E3D5CD8A40BEF38F03B50BB
:107010001D6EDCEF37F0040E3D5CD8A414EF38F0A1
:107020003B501E6EDCEF37F0050E3D5CD8A41DEF23
:1070300038F03B501F6EDCEF37F0060E3D5CD8A4F5
:1070400026EF38F03B50206EDCEF37F0070E3D5C4A
:10705000D8A42FEF38F03B50216EDCEF37F0080E4C
:107060003D5CD8A438EF38F03B50226EDCEF37F0AF
:10707000090E3D5CD8A441EF38F03B50236EDCEFA5
:1070800037F00A0E3D5CD8A44AEF38F03B50246E2E
:10709000DCEF37F00B0E3D5CD8A453EF38F03B50DB
:1070A000256EDCEF37F00C0E3D5CD8A45CEF38F0B9
:1070B0003B50266EDCEF37F00D0E3D5CD8A465EF3B
:1070C00038F03B50276EDCEF37F00E0E3D5CD8A455
:1070D0006EEF38F03B50286EDCEF37F00F0E3D5C62
:1070E000D8A477EF38F03B50296EDCEF37F0100E64
:1070F0003D5CD8A480EF38F03B502A6EDCEF37F0CF
:10710000110E3D5CD8A489EF38F03B502B6EDCEFBC
:1071100037F0120E3D5CD8A492EF38F03B502C6E45
:10712000DCEF37F0130E3D5CD8A49BEF38F03B50FA
:107130002D6EDCEF37F0140E3D5CD8A4A4EF38F0D0
:107140003B502E6EDCEF37F0150E3D5CD8A4ADEF52
:1071500038F03B502F6EDCEF37F0160E3D5CD8A4B4
:10716000B6EF38F03B50306EDCEF37F0170E3D5C79
:10717000D8A4BFEF38F03B50316EDCEF37F0180E7B
:107180003D5CD8A4C8EF38F03B50326EDCEF37F0EE
:10719000190E3D5CD8A4D1EF38F03B50336EDCEFD4
:1071A00037F01A0E3D5CD8A4DAEF38F03B50346E5D
:1071B000DCEF37F01B0E3D5CD8A4E3EF38F03B501A
:1071C000356EDCEF37F01C0E3D5CD8A4ECEF38F0E8
:1071D0003B50366EDCEF37F03B50376E3D6A1200A5
:1071E0001650BF0B616FA80E615DD8B428EF39F05F
:1071F000980E615DD8B42BEF39F0880E615DD8B47C
:107200002EEF39F0619F250E615DD8B431EF39F072
:10721000150E615DD8B434EF39F0050E615DD8B458
:1072200037EF39F0200E615DD8B43AEF39F0100E27
:10723000615DD8B43DEF39F0000E615DD8B440EF28
:1072400039F0300E615DD8B443EF39F046EF39F0D4
:10725000000E47EF39F0010E47EF39F0020E47EF0D
:1072600039F0030E47EF39F0040E47EF39F0050E01
:1072700047EF39F0060E47EF39F0070E47EF39F0C8
:10728000080E47EF39F0090E47EF39F00F0E5D6E2B
:10729000120080BA99EF39F0070E575CD8B454EF5A
:1072A00039F0572A9BEF39F0576A3EBA1200000EA8
:1072B000415CD8B497EF39F0010E415CD8B494EF3B
:1072C00039F0020E415CD8B472EF39F0030E415C24
:1072D000D8B47BEF39F0040E415CD8B484EF39F0B8
:1072E0008DEF39F0466A44A0476A4DAE486A51AE08
:1072F000496A94EF39F0496A43A0466A44A0476A54
:107300004DAE486A94EF39F043A0466A476A4DAEE5
:10731000486A51AE496A94EF39F043A0466A44A0E6
:10732000476A486A51AE496A42EC36F0416A3E8A81
:1073300012003E9A576A12005E0E295CD8B4E4EF40
:1073400039F05D0E295CD8B4E4EF39F0440E295CC5
:10735000D8B4EAEF39F0450E295CD8B4EAEF39F039
:107360003E0E295CD8B4F0EF39F03F0E295CD8B45A
:10737000F0EF39F0220E295CD8B4F6EF39F0230E85
:10738000295CD8B4F6EF39F01F0E295CD8B4FCEFB5
:1073900039F0200E295CD8B4FCEF39F0110E295CCD
:1073A000D8B402EF3AF0120E295CD8B402EF3AF0EA
:1073B000100E295CD8B408EF3AF00F0E295CD8B44F
:1073C00008EF3AF00EEF3AF0010E626F010E636FB4
:1073D00012EF3AF0020E626F010E636F12EF3AF095
:1073E000030E626F010E636F12EF3AF0040E626FCC
:1073F000010E636F12EF3AF0050E626F010E636FBC
:1074000012EF3AF0060E626F020E636F12EF3AF05F
:10741000070E626F020E636F12EF3AF0FE0E626F9C
:10742000030E636F5FA212006351645DD8A41BEF6B
:107430003AF02DEF3AF0010E635DD8B427EF3AF041
:10744000020E635DD8B42AEF3AF02DEF3AF01292B3
:107450002BEF3AF0128292EC36F06351646F120017
:10746000000E405CD8A459EF3AF0AEEC51F0000E9B
:1074700058EC35F01EEC52F0000E58EC35F07EEC76
:1074800051F0000E58EC35F08EEC54F0000E58EC34
:1074900035F08EEC54F0000E58EC35F08EEC54F0D4
:1074A000000E58EC35F08EEC54F0000E58EC35F030
:1074B0001200010E405CD8A482EF3AF08EEC51F03D
:1074C000000E58EC35F00EEC52F0000E58EC35F092
:1074D0003EEC52F0000E58EC35F0BEEC51F0000ED0
:1074E00058EC35F08EEC54F0000E58EC35F08EEC84
:1074F00054F0000E58EC35F08EEC54F0000E58ECC1
:1075000035F01200020E405CD8A4ABEF3AF0CEEC9E
:1075100051F0000E58EC35F01EEC52F0000E58EC15
:1075200035F07EEC52F0000E58EC35F08EEC54F055
:10753000000E58EC35F08EEC54F0000E58EC35F09F
:107540008EEC54F0000E58EC35F08EEC54F0000E3A
:1075500058EC35F01200030E405CD8A4D4EF3AF09A
:107560006EEC51F0000E58EC35F08EEC54F0000E3D
:1075700058EC35F06EEC52F0000E58EC35F07EEC25
:1075800052F0000E58EC35F04EEC51F0000E58EC75
:1075900035F08EEC54F0000E58EC35F08EEC54F0D3
:1075A000000E58EC35F01200040E405CD8A4FDEF3C
:1075B0003AF08EEC52F0000E58EC35F08EEC54F0B0
:1075C000000E58EC35F07EEC51F0000E58EC35F022
:1075D0004EEC51F0000E58EC35F07EEC52F0000EFF
:1075E00058EC35F04EEC51F0000E58EC35F08EECC6
:1075F00054F0000E58EC35F01200050E405CD8A493
:1076000026EF3BF05EEC52F0000E58EC35F08EECBD
:1076100054F0000E58EC35F08EEC51F0000E58ECA2
:1076200035F05EEC52F0000E58EC35F05EEC52F0A6
:10763000000E58EC35F08EEC54F0000E58EC35F09E
:107640008EEC54F0000E58EC35F01200060E405C43
:10765000D8A44FEF3BF01EEC52F0000E58EC35F082
:107660009EEC52F0000E58EC35F08EEC54F0000E0B
:1076700058EC35F08EEC51F0000E58EC35F05EEC25
:1076800052F0000E58EC35F05EEC52F0000E58EC63
:1076900035F08EEC54F0000E58EC35F01200070E69
:1076A000405CD8A478EF3BF05EEC52F0000E58EC52
:1076B00035F06EEC51F0000E58EC35F05EEC51F008
:1076C000000E58EC35F0FEEC51F0000E58EC35F0A1
:1076D0008EEC54F0000E58EC35F08EEC54F0000EA9
:1076E00058EC35F08EEC54F0000E58EC35F01200EA
:1076F000080E405CD8A4A1EF3BF0FEEC4EF0000E6B
:1077000058EC35F0CEEC4EF0000E58EC35F0EEECC7
:1077100051F0000E58EC35F0BEEC51F0000E58EC74
:1077200035F0DEEC52F0000E58EC35F08EEC54F0F3
:10773000000E58EC35F08EEC54F0000E58EC35F09D
:107740001200090E405CD8A4CAEF3BF04EEC51F099
:10775000000E58EC35F08EEC52F0000E58EC35F07F
:107760007EEC51F0000E58EC35F0CEEC51F0000EEE
:1077700058EC35F02EEC52F0000E58EC35F08EEC53
:1077800054F0000E58EC35F08EEC54F0000E58EC2E
:1077900035F012000A0E405CD8A4F3EF3BF09EECEB
:1077A00052F0000E58EC35F0FEEC51F0000E58ECA3
:1077B00035F05EEC52F0000E58EC35F06EEC51F006
:1077C000000E58EC35F0EEEC51F0000E58EC35F0B0
:1077D0008EEC54F0000E58EC35F08EEC54F0000EA8
:1077E00058EC35F012000B0E405CD8A4D5EF3CF0FD
:1077F0007EEC52F0000E58EC35F0BEEC52F0000E6C
:1078000058EC35F08EEC54F0000E58EC35F0155075
:10781000070B406E000E405CD8A424EF3CF05EECF9
:1078200052F0000E58EC35F0BEEC52F0000E58EC61
:1078300035F03EEC52F0000E58EC35F06EEC4EF0A8
:10784000000E58EC35F01200010E405CD8A43EEF5B
:107850003CF05EEC52F0000E58EC35F0BEEC52F00D
:10786000000E58EC35F03EEC52F0000E58EC35F0BE
:107870007EEC4EF0000E58EC35F01200020E405C2B
:10788000D8A458EF3CF05EEC52F0000E58EC35F006
:10789000BEEC52F0000E58EC35F03EEC52F0000E0B
:1078A00058EC35F08EEC4EF0000E58EC35F012002E
:1078B000030E405CD8A472EF3CF08EEC52F0000E48
:1078C00058EC35F06EEC52F0000E58EC35F05EECF2
:1078D00051F0000E58EC35F08EEC54F0000E58ECE0
:1078E00035F01200040E405CD8A48CEF3CF05EEC46
:1078F00052F0000E58EC35F0BEEC52F0000E58EC91
:1079000035F03EEC52F0000E58EC35F0AEEC4EF097
:10791000000E58EC35F01200050E405CD8A4A6EF1E
:107920003CF05EEC52F0000E58EC35F0BEEC52F03C
:10793000000E58EC35F03EEC52F0000E58EC35F0ED
:10794000BEEC4EF0000E58EC35F01200060E405C16
:10795000D8A4C0EF3CF05EEC52F0000E58EC35F0CD
:10796000BEEC52F0000E58EC35F03EEC52F0000E3A
:1079700058EC35F0CEEC4EF0000E58EC35F012001D
:107980005EEC52F0000E58EC35F0BEEC52F0000EFA
:1079900058EC35F03EEC52F0000E58EC35F0DEECD1
:1079A0004EF0000E58EC35F012000C0E405CD8A4DE
:1079B000FEEF3CF09EEC52F0000E58EC35F07EEC01
:1079C00051F0000E58EC35F07EEC51F0000E58EC02
:1079D00035F08EEC54F0000E58EC35F08EEC54F08F
:1079E000000E58EC35F08EEC54F0000E58EC35F0EB
:1079F0008EEC54F0000E58EC35F012000D0E405C89
:107A0000D8A427EF3DF0BEEC51F0000E58EC35F055
:107A10005EEC52F0000E58EC35F00EEC52F0000E19
:107A200058EC35F06EEC51F0000E58EC35F0EEEC01
:107A300051F0000E58EC35F08EEC54F0000E58EC7E
:107A400035F08EEC54F0000E58EC35F012005EEC80
:107A500052F0000E58EC35F08EEC51F0000E58EC60
:107A600035F06EEC52F0000E58EC35F08EEC51F023
:107A7000000E58EC35F05EEC52F0000E58EC35F08C
:107A80009EEC52F0000E58EC35F08EEC51F0000EEA
:107A900058EC35F0120080B067EF3DF0070E565CF1
:107AA000D8B456EF3DF0562A69EF3DF0566A3EB025
:107AB00069EF3DF0000E4A5CD8A463EF3DF0080E7C
:107AC0004A6E64EF3DF04A063E8069EF3DF03E901D
:107AD000566A84B685EF3DF0070E555CD8B474EF56
:107AE0003DF0552A87EF3DF0556A3EBC87EF3DF0EB
:107AF000080E4A5CD8A481EF3DF0000E4A6E82EF7A
:107B00003DF04A2A3E8C87EF3DF03E9C556A1200BC
:107B100080B0A4EF3DF0070E565CD8B493EF3DF073
:107B2000562AA6EF3DF0566A3EB0A6EF3DF0010E94
:107B30004A5CD8A4A0EF3DF0080E4A6EA1EF3DF0DC
:107B40004A063E80A6EF3DF03E90566A84B6C2EFEC
:107B50003DF0070E555CD8B4B1EF3DF0552AC4EFA7
:107B60003DF0556A3EBCC4EF3DF0080E4A5CD8A417
:107B7000BEEF3DF0010E4A6EBFEF3DF04A2A3E8C4B
:107B8000C4EF3DF03E9C556A1200080E4A5CD8B422
:107B9000DCEF3FF03FB40BEF3EF080B8E0EF3DF09C
:107BA000070E585CD8B4D8EF3DF0582AE2EF3DF00C
:107BB000586A3EB89EEF3EF03F843E880BEF3EF0A1
:107BC0003E98586A1AEC35F04D0E26EC35F0BE0E94
:107BD0003FEC35F0000E58EC35F08EEC54F0000E12
:107BE00058EC35F08EEC54F08EEC54F0000E58EC5E
:107BF00035F08EEC54F0000E58EC35F08EEC54F06D
:107C0000000E58EC35F08EEC54F0000E58EC35F0C8
:107C10004B50406E12001AEC35F04D0E26EC35F04C
:107C2000BE0E3FEC35F0000E4A5CD8B438EF3EF0A3
:107C3000010E4A5CD8B43DEF3EF0020E4A5CD8B467
:107C400042EF3EF0030E4A5CD8B447EF3EF0040E1C
:107C50004A5CD8B44CEF3EF0050E4A5CD8B451EF04
:107C60003EF0060E4A5CD8B456EF3EF05BEF3EF0B5
:107C70004CAE60EF3EF080EF3EF04CAC60EF3EF07B
:107C800080EF3EF04CAA60EF3EF080EF3EF04CA853
:107C900060EF3EF080EF3EF04CA660EF3EF080EFEC
:107CA0003EF04CA460EF3EF080EF3EF04CA260EF5F
:107CB0003EF080EF3EF04CA060EF3EF080EF3EF0F3
:107CC000000E58EC35F07EEC4EF0000E58EC35F01E
:107CD0008EEC54F02EEC52F0000E58EC35F05EECC9
:107CE00052F0000E58EC35F08EEC54F0FF0E58ECCC
:107CF00035F00EEC4FF0FF0E58EC35F09EEF3EF0F5
:107D0000FF0E58EC35F01EEC4FF0FF0E58EC35F03E
:107D10008EEC54F02EEC52F0000E58EC35F05EEC88
:107D200052F0000E58EC35F08EEC54F0000E58EC8A
:107D300035F06EEC4EF0000E58EC35F04B50406EC6
:107D40003FA4120080BAB7EF3EF0070E575CD8B4DC
:107D5000ADEF3EF0572AB9EF3EF0576A3EBAB9EFA1
:107D60003EF03F944B50406E4C6E3E8A12003E9A5D
:107D7000576A80B83BEF3FF0070E585CD8B4C4EFA9
:107D80003EF0582A3DEF3FF0586A3EB83DEF3FF0D5
:107D9000000E4A5CD8B4EDEF3EF0010E4A5CD8B458
:107DA000F6EF3EF0020E4A5CD8B4FFEF3EF0030E51
:107DB0004A5CD8B408EF3FF0040E4A5CD8B411EF27
:107DC0003FF0050E4A5CD8B41AEF3FF0060E4A5C4D
:107DD000D8B423EF3FF02CEF3FF04CAEF3EF3EF082
:107DE0004B8E35EF3FF04B9E35EF3FF04CACFCEF48
:107DF0003EF04B8C35EF3FF04B9C35EF3FF04CAAFB
:107E000005EF3FF04B8A35EF3FF04B9A35EF3FF0EF
:107E10004CA80EEF3FF04B8835EF3FF04B9835EF15
:107E20003FF04CA617EF3FF04B8635EF3FF04B96F7
:107E300035EF3FF04CA420EF3FF04B8435EF3FF09F
:107E40004B9435EF3FF04CA229EF3FF04B8235EFDA
:107E50003FF04B9235EF3FF04CA032EF3FF04B80BC
:107E600035EF3FF04B9035EF3FF03F944B50406E75
:107E70003E883DEF3FF03E98586A80B08AEF3FF071
:107E8000070E565CD8B448EF3FF0562A8CEF3FF00F
:107E9000566A3EB08CEF3FF0000E4A5CD8B471EFEA
:107EA0003FF0010E4A5CD8B474EF3FF0020E4A5C1A
:107EB000D8B477EF3FF0030E4A5CD8B47AEF3FF0C6
:107EC000040E4A5CD8B47DEF3FF0050E4A5CD8B48E
:107ED00080EF3FF0060E4A5CD8B483EF3FF086EFA8
:107EE0003FF04C7E87EF3FF04C7C87EF3FF04C7AC1
:107EF00087EF3FF04C7887EF3FF04C7687EF3FF00D
:107F00004C7487EF3FF04C7287EF3FF04C703E802F
:107F10008CEF3FF03E90566A84B6D9EF3FF0070EE3
:107F2000555CD8B497EF3FF0552ADCEF3FF0556A27
:107F30003EBCDBEF3FF0000E4A5CD8B4C0EF3FF030
:107F4000010E4A5CD8B4C3EF3FF0020E4A5CD8B4CD
:107F5000C6EF3FF0030E4A5CD8B4C9EF3FF0040E01
:107F60004A5CD8B4CCEF3FF0050E4A5CD8B4CFEFF2
:107F70003FF0060E4A5CD8B4D2EF3FF0D5EF3FF0A9
:107F80004C7ED6EF3FF04C7CD6EF3FF04C7AD6EFEC
:107F90003FF04C78D6EF3FF04C76D6EF3FF04C7484
:107FA000D6EF3FF04C72D6EF3FF04C703E8CDBEFDB
:107FB0003FF03E9C556A120080B85AEF40F0070E21
:107FC000585CD8B4E7EF3FF0582A5CEF40F0586AAD
:107FD0003EB85CEF40F0000E465CD8B41EEF40F0B7
:107FE000010E465CD8B422EF40F0020E465CD8B4D5
:107FF00026EF40F0030E465CD8B42AEF40F0040EA2
:10800000465CD8B42EEF40F0050E465CD8B432EF93
:1080100040F0060E465CD8B43AEF40F0070E465CDE
:10802000D8B43EEF40F0080E465CD8B442EF40F0C2
:10803000090E465CD8B446EF40F012004B50116E6A
:1080400048EF40F04B50126E48EF40F04B50136E2B
:1080500048EF40F04B50146E48EF40F04B50156E17
:1080600048EF40F04B50166EF0EC38F05D505E6E0D
:1080700048EF40F04B50176E48EF40F04B50186EF1
:1080800048EF40F04B50196E48EF40F04B501A6EDD
:108090005FEC36F04B50406E3E88000E465CD8B424
:1080A00056EF40F0070E4A6E5CEF40F0050E4A6E48
:1080B0005CEF40F03E98586A12001AEC35F0670EFB
:1080C00026EC35F0BC0E3FEC35F03FBC7CEF40F0C9
:1080D000000E58EC35F0CEEC52F0000E58EC35F0B6
:1080E0008EEC51F0000E58EC35F06EEC52F0000EB4
:1080F00058EC35F08EEF40F0FF0E58EC35F06EEC9A
:1081000054F0FF0E58EC35F02EEC53F0FF0E58EC07
:1081100035F00EEC54F0FF0E58EC35F01DEC35F058
:10812000440E26EC35F0BC0E3FEC35F03FBCADEF15
:1081300040F0FF0E58EC35F0BEEC53F0FF0E58EC5B
:1081400035F09EEC54F0FF0E58EC35F0CEEC53F0C9
:10815000FF0E58EC35F0BFEF40F0000E58EC35F054
:108160001EEC52F0000E58EC35F08EEC54F0000E80
:1081700058EC35F02EEC52F0000E58EC35F080B093
:10818000D8EF40F0070E565CD8B4CAEF40F0562A3C
:10819000DAEF40F0566A3EB0DAEF40F03FBCD4EF81
:1081A00040F03F8CD5EF40F03F9C3E80DAEF40F04E
:1081B0003E90566A84B6F3EF40F0070E555CD8B493
:1081C000E5EF40F0552AF5EF40F0556A3EBCF5EF7B
:1081D00040F03FBCEFEF40F03F8CF0EF40F03F9CB1
:1081E0003E8CF5EF40F03E9C556A120080B877EF68
:1081F00041F0070E585CD8B401EF41F0582A79EFEE
:1082000041F0586A3EB879EF41F03FAC6FEF41F072
:1082100042EC36F0000E475CD8B443EF41F0010E5B
:10822000475CD8B447EF41F0020E475CD8B44BEF3F
:1082300041F0030E475CD8B44FEF41F0040E475CA9
:10824000D8B453EF41F0050E475CD8B457EF41F076
:10825000060E475CD8B45BEF41F0070E475CD8B41C
:108260005FEF41F0080E475CD8B463EF41F0090EB0
:10827000475CD8B467EF41F00A0E475CD8B46BEFA7
:1082800041F06FEF41F026EC55F06FEF41F039EC23
:1082900055F06FEF41F04CEC55F06FEF41F05FECB3
:1082A00055F06FEF41F072EC55F06FEF41F085EC57
:1082B00055F06FEF41F098EC55F06FEF41F0ABECFB
:1082C00055F06FEF41F0BEEC55F06FEF41F0D1EC9F
:1082D00055F06FEF41F0E4EC55F0F8EC55F042EC5E
:1082E00036F0446A476A3F9C3E8842EF01F03E9870
:1082F000586A120083A29AEF41F03FB812004DB2C3
:108300008CEF41F01550380B406E180E406E155032
:10831000C70B156E94EF41F015503F0B406E1B0ECE
:10832000406E1550C00B156E405015125FEC36F0C4
:108330003F8812003F9812001550380B406E4042A3
:10834000404240424050070B406E1550F80B156EEE
:10835000405015121200106E000E105CD8A4C9EF28
:1083600041F005B8BAEF41F005BABEEF41F0CEECEE
:108370004DF012008EEC54F0058C120005BCC5EFD8
:1083800041F0059CCEEC4DF01200059C8EEC54F0B3
:108390001200010E105CD8A4D1EF41F0DEEC4DF0DC
:1083A0001200020E105CD8A4D9EF41F0EEEC4DF0B3
:1083B0001200030E105CD8A4E1EF41F0FEEC4DF08A
:1083C0001200040E105CD8A4E9EF41F00EEC4EF060
:1083D0001200050E105CD8A4F1EF41F01EEC4EF037
:1083E0001200060E105CD8A4F9EF41F02EEC4EF00E
:1083F0001200070E105CD8A401EF42F03EEC4EF0E4
:108400001200080E105CD8A409EF42F04EEC4EF0BA
:1084100012005EEC4EF01200106E000E105CD8A43C
:1084200015EF42F06EEC4EF01200010E105CD8A475
:108430001DEF42F07EEC4EF01200020E105CD8A44C
:1084400025EF42F08EEC4EF01200030E105CD8A423
:108450002DEF42F09EEC4EF01200040E105CD8A4FA
:1084600035EF42F0AEEC4EF01200050E105CD8A4D1
:108470003DEF42F0BEEC4EF01200060E105CD8A4A8
:1084800045EF42F0CEEC4EF01200070E105CD8A47F
:108490004DEF42F0DEEC4EF01200080E105CD8A456
:1084A00055EF42F0EEEC4EF01200FEEC4EF01200F2
:1084B000106E000E105CD8A461EF42F00EEC4FF08D
:1084C0001200010E105CD8A469EF42F01EEC4FF0D0
:1084D0001200020E105CD8A471EF42F02EEC4FF0A7
:1084E0001200030E105CD8A479EF42F03EEC4FF07E
:1084F0001200040E105CD8A481EF42F04EEC4FF055
:108500001200050E105CD8A489EF42F05EEC4FF02B
:108510001200060E105CD8A491EF42F06EEC4FF002
:108520001200070E105CD8A499EF42F07EEC4FF0D9
:108530001200080E105CD8A4A1EF42F08EEC4FF0B0
:1085400012009EEC4FF01200062A0A0E065CD8A418
:10855000A4EF42F0066A1200062AFF0E065CD8A4B9
:10856000ACEF42F0066A072A640E075CD8A4ACEFB1
:1085700042F0066A076A1200062AFF0E065CD8A4BB
:10858000BCEF42F0066A072AFF0E075CD8A4BCEFD6
:1085900042F0066A076A12001AEC35F0400E26EC2B
:1085A00035F0BF0E3FEC35F07EEC51F0000E58EC8C
:1085B00035F04EEC51F0000E58EC35F0CEEC51F0A9
:1085C000000E58EC35F0EEEC4EF0000E58EC35F0A5
:1085D000AEEC4EF0000E58EC35F07EEC4EF0000E96
:1085E00058EC35F0CEEC4EF08EEC54F05EEC52F0E0
:1085F000000E58EC35F08EEC51F0000E58EC35F0D2
:108600009EEC52F01DEC35F0400E26EC35F0BF0E1E
:108610003FEC35F0400E58EC35F0000E58EC35F0DC
:108620006EEC4EF0000E58EC35F08EEC54F0EEECA3
:1086300051F0000E58EC35F04EEC51F0000E58ECB5
:1086400035F0CEEC51F0000E58EC35F0400E036ED4
:108650007F0E046E1AEC35F0035026EC35F0BC0E9C
:108660003FEC35F0010E58EC35F01DEC35F00450C0
:1086700026EC35F0BC0E3FEC35F0010E58EC35F031
:10868000032A0406ACEC42F0800E035CD8A42AEF67
:1086900043F0BCEC42F0BCEC42F0BCEC42F0BCEC71
:1086A00042F0BCEC42F0400E036E7F0E046E1AECFA
:1086B00035F0035026EC35F0BC0E3FEC35F0000EE3
:1086C00058EC35F01DEC35F0045026EC35F0BC0EBE
:1086D0003FEC35F0000E58EC35F0032A0406ACEC04
:1086E00042F0800E035CD8A457EF43F03F8EBCEC01
:1086F00042F0BCEC42F0BCEC42F0BCEC42F05180E9
:108700001AEC35F04A0E26EC35F0BB0E3FEC35F096
:10871000FEEC4FF0000E58EC35F0100E58EC35F032
:10872000100E58EC35F0100E58EC35F0100E58ECD9
:1087300035F0100E58EC35F0000E58EC35F07EECAC
:1087400050F0000E58EC35F08EEC54F0000E58EC62
:1087500035F0EEEC4FF0000E58EC35F07EEC50F0BA
:10876000000E58EC35F00EEC50F0000E58EC35F0E1
:108770002EEC50F0000E58EC35F07EEC50F0000E70
:1087800058EC35F01DEC35F0400E26EC35F0BB0E04
:108790003FEC35F0EEEC4FF0000E58EC35F0EEEC1F
:1087A0004FF0000E58EC35F0BEEC50F0000E58ECD7
:1087B00035F02EEC50F0000E58EC35F07EEC50F019
:1087C000000E58EC35F00EEC50F0000E58EC35F081
:1087D00051901AEC35F0560E26EC35F0BC0E3FECFD
:1087E00035F0AEEC4FF0000E58EC35F0EEEC50F0FA
:1087F000000E58EC35F0DEEC4FF0000E58EC35F082
:108800002EEC50F0000E58EC35F08EEC50F0000ECF
:1088100058EC35F08EEC54F0000E58EC35F05EEC70
:1088200050F0000E58EC35F01DEC35F0400E26EC03
:1088300035F0BC0E3FEC35F0AEEC4FF0000E58ECCE
:1088400035F0BEEC4FF0000E58EC35F08EEC50F0E9
:10885000000E58EC35F0BEEC50F0000E58EC35F040
:10886000AEEC4FF0000E58EC35F0DEEC50F0000EA0
:1088700058EC35F08EEC50F0000E58EC35F0BEECB4
:1088800050F0000E58EC35F02EEC51F0000E58EC84
:1088900035F0522A080E525CD8A477EF43F03F9E81
:1088A000526ABCEC42F0BCEC42F0BCEC42F0BCECD6
:1088B00042F0BCEC42F0BCEC42F0BCEC42F0BCEC50
:1088C00042F0BCEC42F0BCEC42F0BCEC42F0BCEC40
:1088D00042F0BCEC42F0BCEC42F0BCEC42F0BCEC30
:1088E00042F0BCEC42F0BCEC42F0BCEC42F0BCEC20
:1088F00042F0BCEC42F0BCEC42F0BCEC42F0BCEC10
:1089000042F0BCEC42F0BCEC42F0BCEC42F0BCECFF
:1089100042F0BCEC42F0BCEC42F0BCEC42F0BCECEF
:1089200042F0BCEC42F0BCEC42F0BCEC42F0BCECDF
:1089300042F0BCEC42F0BCEC42F0BCEC42F0BCECCF
:1089400042F0BCEC42F0BCEC42F0BCEC42F0BCECBF
:1089500042F0BCEC42F0BCEC42F0BCEC42F0BCECAF
:1089600042F0BCEC42F0BCEC42F0BCEC42F0BCEC9F
:1089700042F0BCEC42F0BCEC42F0BCEC42F0BCEC8F
:1089800042F0BCEC42F0BCEC42F0BCEC42F0BCEC7F
:1089900042F0BCEC42F0BCEC42F0BCEC42F0BCEC6F
:1089A00042F0BCEC42F0BCEC42F0BCEC42F0BCEC5F
:1089B00042F0BCEC42F0BCEC42F0BCEC42F0BCEC4F
:1089C00042F0BCEC42F0BCEC42F042EC36F0BCECC5
:1089D00042F0BCEC42F0BCEC42F0BCEC42F01200C5
:1089E00016AEF6EF44F06687F7EF44F0669716ACE4
:1089F000FEEF44F06597658500EF45F06597659556
:108A000016AA05EF45F012EF45F016A80DEF45F058
:108A1000659F658D659B1DEF45F0659F659D659B19
:108A20001DEF45F016A81AEF45F0658F658D658B33
:108A30001DEF45F0658F659D659B16A623EF45F0FC
:108A4000659924EF45F0658916A42AEF45F0658104
:108A50002BEF45F0659116A031EF45F0658332EFBD
:108A600045F065935FA038EF45F0678F39EF45F02B
:108A7000679F1200D40E51EC45F0000E51EC45F00A
:108A8000020E51EC45F0625151EC45F0655151EC4C
:108A900045F0665151EC45F0675151EC45F08C863C
:108AA00012003C6E8C963CB059EF45F08B985AEF13
:108AB00045F08B888C84000000000000000000005E
:108AC0000000000000008C94000000000000000086
:108AD00000000000000000003A2A3C42080E3A5C08
:108AE000D8A453EF45F03A6A1200096E640E095E8D
:108AF000D8A07EEF45F00A2A76EF45F0640E0926ED
:108B00000A0E095ED8A088EF45F00B2A80EF45F0E9
:108B10000A0E0926010E095ED8A092EF45F00C2A34
:108B20008AEF45F012000D6E100E0D5ED8A09CEF7E
:108B300045F00B2A94EF45F0100E0D26010E0D5E48
:108B4000D8A0A6EF45F00C2A9EEF45F0120005884C
:108B50000A50ABEC41F0000E58EC35F00598058A50
:108B60000B50ABEC41F0000E58EC35F0059A0C5070
:108B7000ABEC41F0000E58EC35F00A6A0B6A0C6A57
:108B800012000A500CEC42F0000E58EC35F00B507D
:108B90000CEC42F0000E58EC35F00C500CEC42F0AE
:108BA000000E58EC35F00A6A0B6A0C6A12000A5083
:108BB00058EC42F0FF0E58EC35F00B5058EC42F0F8
:108BC000FF0E58EC35F00C5058EC42F0FF0E58EC0C
:108BD00035F00A6A0B6A0C6A1200406E452A090ECB
:108BE000455CD8B403EF46F040BEFBEF45F06EECB9
:108BF0004EF0FDEF45F07EEC4EF0000E58EC35F0F7
:108C00004046EEEF45F0456A1200406E080E455CA6
:108C1000D8B442EF46F040BE27EF46F045504A5CDC
:108C2000D8B41DEF46F0000E58EC35F06EEC4EF067
:108C3000000E58EC35F03EEF46F0FF0E58EC35F0E4
:108C40000EEC4FF0FF0E58EC35F03EEF46F045507D
:108C50004A5CD8B436EF46F0000E58EC35F07EECA6
:108C60004EF0000E58EC35F03EEF46F0FF0E58EC9B
:108C700035F01EEC4FF0FF0E58EC35F0452A40461B
:108C800006EF46F0456A12007D0E505CD8B44BEFFB
:108C900046F0502A12003F8A506A12001DEC35F04F
:108CA000530E26EC35F0BE0E3FEC35F0080E4A5C54
:108CB000D8A4A6EF46F0FF0E58EC35F00EEC54F0B9
:108CC000FF0E58EC35F02EEC53F0FF0E58EC35F05B
:108CD0001EEC54F0FF0E58EC35F01AEC35F0460E51
:108CE00026EC35F0BC0E3FEC35F0000E58EC35F0BC
:108CF0008EEC54F0000E58EC35F08EEC54F0000E73
:108D000058EC35F08EEC54F0000E58EC35F08EEC4B
:108D100054F0000E58EC35F08EEC54F0000E58EC88
:108D200035F08EEC54F0000E58EC35F08EEC54F02B
:108D3000000E58EC35F08EEC54F0000E58EC35F087
:108D40008EEC54F0000E58EC35F01200000E58EC8A
:108D500035F06EEC52F0000E58EC35F08EEC51F020
:108D6000000E58EC35F07EEC52F0000E58EC35F069
:108D700012001DEC35F0400E26EC35F0BB0E3FEC3A
:108D800035F01200000E58EC35F01EEC52F0000EDB
:108D900058EC35F02EEC52F0000E58EC35F08EEC1D
:108DA00054F0000E58EC35F044EC48F08EEC54F0E2
:108DB000000E58EC35F08EEC54F08EEC54F09FEC35
:108DC00048F01200FF0E58EC35F0EEEC53F0FF0EB9
:108DD00058EC35F00EEC53F0FF0E58EC35F0FEEC8D
:108DE00053F0FF0E58EC35F00EEC53F0FF0E58EC3C
:108DF00035F09EEC54F0FF0E58EC35F05EEC48F088
:108E00009FEC48F01200FF0E58EC35F00EEC53F0DA
:108E1000FF0E58EC35F00EEC53F0FF0E58EC35F029
:108E2000FEEC53F0FF0E58EC35F00EEC53F0FF0E55
:108E300058EC35F09EEC54F0FF0E58EC35F05EEC3B
:108E400048F09FEC48F01200FF0E58EC35F02EEC85
:108E500054F0FF0E58EC35F0BEEC53F0FF0E58EC1A
:108E600035F09EEC53F0FF0E58EC35F0CEEC53F09D
:108E7000FF0E58EC35F00EEC53F0FF0E58EC35F0C9
:108E80008EEC53F0FF0E58EC35F08EEC54F0000EE3
:108E900058EC35F08EEC54F0000E58EC35F08EECBA
:108EA00054F0000E58EC35F08EEC54F0000E58ECF7
:108EB00035F09FEC48F01200FF0E58EC35F03EEC18
:108EC00054F0FF0E58EC35F0EEEC52F0FF0E58EC7B
:108ED00035F09EEC53F0FF0E58EC35F06EEC53F08D
:108EE000FF0E58EC35F01EEC53F0FF0E58EC35F049
:108EF0006EEC53F0FF0E58EC35F01EEC54F0FF0E04
:108F000058EC35F06EEC54F0FF0E58EC35F09EEC5A
:108F100054F02EEC53F0FF0E58EC35F0810E58EC67
:108F200035F0ED0E58EC35F0ED0E58EC35F0ED0E59
:108F300058EC35F0B9EC46F0930E58EC35F0FF0ED6
:108F400058EC35F068EC48F08EEC54F0000E58EC1C
:108F500035F01200FF0E58EC35F0FEEC52F0FF0E2B
:108F600058EC35F06EEC53F0FF0E58EC35F09EECFB
:108F700054F0FF0E58EC35F0DEEC53F0FF0E58ECD9
:108F800035F05EEC53F0FF0E58EC35F0EEEC52F09D
:108F9000FF0E58EC35F00EEC54F0FF0E58EC35F0A7
:108FA0002EEC53F0FF0E58EC35F09EEC54F02EEC06
:108FB00053F0FF0E58EC35F0810E58EC35F0ED0E05
:108FC00058EC35F0ED0E58EC35F0ED0E58EC35F070
:108FD000B9EC46F0930E58EC35F0FF0E58EC35F036
:108FE00068EC48F08EEC54F0000E58EC35F01200AE
:108FF000FF0E58EC35F0DEEC53F0FF0E58EC35F078
:10900000EEEC52F0FF0E58EC35F0FEEC53F0FF0E94
:1090100058EC35F06EEC53F0FF0E58EC35F01EECCA
:1090200054F0FF0E58EC35F06EEC54F0FF0E58EC97
:1090300035F09EEC54F02EEC53F0FF0E58EC35F06A
:10904000FEEC53F0FF0E58EC35F0FEEC53F0FF0E43
:1090500058EC35F0C30E58EC35F0BD0E58EC35F039
:10906000BD0E58EC35F0BD0E58EC35F0B9EC46F0BD
:10907000C30E58EC35F0FF0E58EC35F072EC48F0AA
:10908000000E58EC35F012008EEC51F0000E58EC4A
:1090900035F05EEC52F0000E58EC35F05EEC52F01C
:1090A000000E58EC35F02EEC52F0000E58EC35F076
:1090B0005EEC52F0000E58EC35F012002EEC53F03E
:1090C000FF0E58EC35F0FEEC53F0FF0E58EC35F087
:1090D000FEEC53F0FF0E58EC35F0CEEC53F0FF0EE3
:1090E00058EC35F0FEEC53F0FF0E58EC35F0120062
:1090F0005EEC48F09EEC54F0FF0E58EC35F00EECB0
:1091000053F0FF0E58EC35F0CEEC53F0FF0E58EC58
:1091100035F01EEC53F0FF0E58EC35F02EEC53F00A
:10912000FF0E58EC35F0FF0E58EC35F0FF0E58EC02
:1091300035F0FF0E58EC35F0B9EC46F01200B9EC02
:1091400046F08EEC54F0000E58EC35F08EEC54F0F6
:10915000000E58EC35F08EEC54F0000E58EC35F063
:109160008EEC54F0000E58EC35F08EEC54F0000EFE
:1091700058EC35F012006EEC51F0000E58EC35F062
:109180002EEC52F0000E58EC35F01EEC52F0000EB2
:1091900058EC35F07EEC52F0000E58EC35F05EECF9
:1091A00052F0000E58EC35F02EEC52F0000E58EC58
:1091B00035F0FEEC51F0000E58EC35F08EEC54F02A
:1091C0006EEC4EF0000E58EC35F08EEC54F01DECC9
:1091D00035F0400E26EC35F0B90E3FEC35F0FF0EC1
:1091E00058EC35F0810E58EC35F0810E58EC35F026
:1091F000000E58EC35F06EEC4EF0000E58EC35F0E9
:109200006EEC4EF0000E58EC35F0BEEC51F0000E56
:1092100058EC35F0810E58EC35F0810E58EC35F0F5
:10922000FF0E58EC35F012006EEC51F0000E58ECC9
:1092300035F02EEC52F0000E58EC35F01EEC52F0EA
:10924000000E58EC35F07EEC52F0000E58EC35F084
:109250005EEC52F0000E58EC35F02EEC52F0000EA1
:1092600058EC35F0FEEC51F0000E58EC35F08EEC79
:1092700054F07EEC4EF0000E58EC35F08EEC54F0CD
:109280001DEC35F0400E26EC35F0B90E3FEC35F014
:10929000FF0E58EC35F0810E58EC35F0810E58EC8D
:1092A00035F0000E58EC35F06EEC4EF0000E58EC38
:1092B00035F07EEC4EF0000E58EC35F0BEEC51F07F
:1092C000000E58EC35F0810E58EC35F0810E58EC5C
:1092D00035F0FF0E58EC35F012006EEC51F0000E38
:1092E00058EC35F02EEC52F0000E58EC35F01EEC38
:1092F00052F0000E58EC35F07EEC52F0000E58ECB7
:1093000035F05EEC52F0000E58EC35F02EEC52F0D9
:10931000000E58EC35F0FEEC51F0000E58EC35F034
:109320008EEC54F08EEC4EF0000E58EC35F08EECD6
:1093300054F01DEC35F0400E26EC35F0B90E3FEC44
:1093400035F0FF0E58EC35F0810E58EC35F0810EFB
:1093500058EC35F0000E58EC35F06EEC4EF0000E87
:1093600058EC35F08EEC4EF0000E58EC35F0BEECBB
:1093700051F0000E58EC35F0810E58EC35F0810EAE
:1093800058EC35F0FF0E58EC35F012006EEC51F051
:10939000000E58EC35F02EEC52F0000E58EC35F083
:1093A0001EEC52F0000E58EC35F07EEC52F0000E40
:1093B00058EC35F05EEC52F0000E58EC35F02EEC27
:1093C00052F0000E58EC35F0FEEC51F0000E58EC67
:1093D00035F08EEC54F09EEC4EF0000E58EC35F06B
:1093E0008EEC54F01DEC35F0400E26EC35F0B90E45
:1093F0003FEC35F0FF0E58EC35F0810E58EC35F0AF
:10940000810E58EC35F0000E58EC35F06EEC4EF055
:10941000000E58EC35F09EEC4EF0000E58EC35F096
:10942000BEEC51F0000E58EC35F0810E58EC35F0E2
:10943000810E58EC35F0FF0E58EC35F012006EEC52
:1094400051F0000E58EC35F02EEC52F0000E58ECB6
:1094500035F01EEC52F0000E58EC35F07EEC52F078
:10946000000E58EC35F05EEC52F0000E58EC35F082
:109470002EEC52F0000E58EC35F0FEEC51F0000EE0
:1094800058EC35F08EEC54F0AEEC4EF0000E58EC8B
:1094900035F08EEC54F01DEC35F0400E26EC35F036
:1094A000B90E3FEC35F0FF0E58EC35F0810E58EC5C
:1094B00035F0810E58EC35F0000E58EC35F06EECBE
:1094C0004EF0000E58EC35F0AEEC4EF0000E58ECBD
:1094D00035F0BEEC51F0000E58EC35F0810E58EC32
:1094E00035F0810E58EC35F0FF0E58EC35F01200D7
:1094F0006EEC52F0000E58EC35F08EEC51F0000E90
:1095000058EC35F05EEC52F0000E58EC35F0CEEC35
:1095100051F0000E58EC35F04EEC51F0000E58ECC6
:1095200035F0FEEC51F0000E58EC35F08EEC54F0B6
:109530004EEC51F0000E58EC35F08EEC52F0000E6F
:1095400058EC35F07EEC51F01DEC35F0400E26EC79
:1095500035F0B90E3FEC35F0000E58EC35F0CEEC9E
:1095600051F0000E58EC35F02EEC52F0000E58EC95
:1095700035F01AEC35F04C0E26EC35F0BA0E3FEC17
:1095800035F07EEC51F0000E58EC35F04EEC51F019
:10959000000E58EC35F07EEC52F0000E58EC35F031
:1095A0004EEC51F0000E58EC35F08EEC54F09EEC81
:1095B00051F0000E58EC35F02EEC52F0000E58EC45
:1095C00035F05EEC52F0000E58EC35F00EEC52F037
:1095D0001DEC35F0400E26EC35F0BA0E3FEC35F0C0
:1095E000000E58EC35F04EEC51F0000E58EC35F012
:1095F0007EEC52F08EEC54F0FF0E58EC35F0810EFC
:1096000058EC35F0810E58EC35F0000E58EC35F082
:109610006EEC4EF0000E58EC35F0BEEC4EF0000E45
:1096200058EC35F0BEEC51F0000E58EC35F0810EE0
:1096300058EC35F0810E58EC35F0FF0E58EC35F053
:1096400012005EEC52F0000E58EC35F08EEC51F04A
:10965000000E58EC35F06EEC51F0000E58EC35F081
:109660008EEC51F0000E58EC35F0CEEC51F0000EBF
:1096700058EC35F09EEC52F0000E58EC35F08EECC4
:1096800051F0000E58EC35F05EEC52F0000E58EC44
:1096900035F08EEC54F08EEC51F01DEC35F0400EB0
:1096A00026EC35F0B90E3FEC35F0000E58EC35F0F5
:1096B0005EEC52F0000E58EC35F05EEC52F0000E0D
:1096C00058EC35F02EEC52F0000E58EC35F05EEC14
:1096D00052F0000E58EC35F08EEC54F00EEC52F0D7
:1096E000000E58EC35F04EEC51F0000E58EC35F011
:1096F0006EEC52F0000E58EC35F0EEEC51F0000E2E
:1097000058EC35F01DEC35F0640E26EC35F0BA0E51
:109710003FEC35F0FF0E58EC35F0810E58EC35F08B
:10972000810E58EC35F0000E58EC35F06EEC4EF032
:10973000000E58EC35F0CEEC4EF0000E58EC35F043
:10974000BEEC51F0000E58EC35F0810E58EC35F0BF
:10975000810E58EC35F0FF0E58EC35F01200CEECCF
:1097600051F0000E58EC35F01EEC52F0000E58ECA3
:1097700035F07EEC52F0000E58EC35F08EEC51F0E6
:10978000000E58EC35F05EEC52F0000E58EC35F05F
:109790005EEC52F0000E58EC35F08EEC52F0000EFC
:1097A00058EC35F03EEC52F0000E58EC35F07EEC03
:1097B00052F08EEC54F01DEC35F0400E26EC35F0F6
:1097C000B90E3FEC35F0000E58EC35F00EEC52F0CF
:1097D000000E58EC35F04EEC51F0000E58EC35F020
:1097E0006EEC52F0000E58EC35F0EEEC51F08EECD1
:1097F00054F0FF0E58EC35F0810E58EC35F0810E28
:1098000058EC35F0000E58EC35F06EEC4EF0000ED2
:1098100058EC35F0DEEC4EF0000E58EC35F0BEECB6
:1098200051F0000E58EC35F0810E58EC35F0810EF9
:1098300058EC35F0FF0E58EC35F01200CEEC51F03C
:10984000000E58EC35F01EEC52F0000E58EC35F0DE
:109850007EEC52F0000E58EC35F08EEC51F0000E1C
:1098600058EC35F05EEC52F0000E58EC35F05EEC42
:1098700052F0000E58EC35F08EEC52F0000E58EC21
:1098800035F03EEC52F0000E58EC35F07EEC52F024
:109890008EEC54F01DEC35F0400E26EC35F0B90E90
:1098A0003FEC35F0000E58EC35F00EEC52F0000EA7
:1098B00058EC35F02EEC52F0000E58EC35F07EEC02
:1098C00051F0000E58EC35F08EEC51F0000E58ECD3
:1098D00035F08EEC54F00EEC52F0000E58EC35F0F2
:1098E0006EEC52F0000E58EC35F05EEC51F0000ECC
:1098F00058EC35F01DEC35F0640E26EC35F0BA0E60
:109900003FEC35F0FF0E58EC35F0810E58EC35F099
:10991000810E58EC35F0000E58EC35F06EEC4EF040
:10992000000E58EC35F0EEEC4EF0000E58EC35F031
:10993000BEEC51F0000E58EC35F0810E58EC35F0CD
:10994000810E58EC35F0FF0E58EC35F01200CEECDD
:1099500051F0000E58EC35F01EEC52F0000E58ECB1
:1099600035F07EEC52F0000E58EC35F08EEC51F0F4
:10997000000E58EC35F05EEC52F0000E58EC35F06D
:109980005EEC52F0000E58EC35F08EEC52F0000E0A
:1099900058EC35F03EEC52F0000E58EC35F07EEC11
:1099A00052F08EEC54F01DEC35F0400E26EC35F004
:1099B000B90E3FEC35F0000E58EC35F00EEC52F0DD
:1099C000000E58EC35F02EEC52F0000E58EC35F04D
:1099D0007EEC51F0000E58EC35F08EEC51F0000E9C
:1099E00058EC35F08EEC54F0FEEC51F0000E58ECD3
:1099F00035F06EEC52F0000E58EC35F05EEC51F0A4
:109A0000000E58EC35F01DEC35F0640E26EC35F008
:109A1000BA0E3FEC35F0FF0E58EC35F0810E58ECE5
:109A200035F0810E58EC35F0000E58EC35F06EEC48
:109A30004EF0000E58EC35F0FEEC4EF0000E58ECF7
:109A400035F0BEEC51F0000E58EC35F0810E58ECBC
:109A500035F0810E58EC35F0FF0E58EC35F0120061
:109A6000FF0E58EC35F0DEEC53F0FF0E58EC35F0FD
:109A70000EEC53F0FF0E58EC35F00EEC53F0FF0EE9
:109A800058EC35F05EEC53F0FF0E58EC35F0120058
:109A9000FF0E58EC35F0CEEC53F0FF0E58EC35F0DD
:109AA0000EEC54F0FF0E58EC35F09EEC53F0FF0E28
:109AB00058EC35F06EEC53F0FF0E58EC35F0DEEC60
:109AC00053F0FF0E58EC35F01200FF0E58EC35F055
:109AD0001EEC53F0FF0E58EC35F02EEC53F0FF0E59
:109AE00058EC35F01EEC54F0FF0E58EC35F00EEC4F
:109AF00053F0FF0E58EC35F01200FF0E58EC35F025
:109B00000EEC53F0FF0E58EC35F00EEC53F0FF0E58
:109B100058EC35F05EEC53F0FF0E58EC35F01200C7
:109B2000FF0E58EC35F0FEEC53F0FF0E58EC35F01C
:109B30002EEC53F0FF0E58EC35F0FEEC53F0FF0E18
:109B400058EC35F0FEEC53F0FF0E58EC35F01200F7
:109B5000FF0E58EC35F0EEEC53F0FF0E58EC35F0FC
:109B60000EEC53F0FF0E58EC35F05EEC53F0FF0EA8
:109B700058EC35F01200FF0E58EC35F03EEC53F087
:109B8000FF0E58EC35F00EEC53F0FF0E58EC35F0AC
:109B90005EEC53F0FF0E58EC35F012007C0E58ECE2
:109BA00035F0820E58EC35F0820E58EC35F0820E0E
:109BB00058EC35F07C0E58EC35F01200000E58ECE5
:109BC00035F0840E58EC35F0FE0E58EC35F0800E72
:109BD00058EC35F0000E58EC35F01200E20E58EC5F
:109BE00035F0920E58EC35F0920E58EC35F0920E9E
:109BF00058EC35F08C0E58EC35F01200440E58EC51
:109C000035F0820E58EC35F0920E58EC35F0920E8D
:109C100058EC35F06C0E58EC35F01200300E58EC64
:109C200035F0280E58EC35F0240E58EC35F0FE0EC9
:109C300058EC35F0200E58EC35F012004E0E58EC72
:109C400035F08A0E58EC35F08A0E58EC35F08A0E55
:109C500058EC35F0720E58EC35F012007C0E58ECD2
:109C600035F0920E58EC35F0920E58EC35F0920E1D
:109C700058EC35F0640E58EC35F01200060E58EC36
:109C800035F0020E58EC35F0C20E58EC35F0320EBD
:109C900058EC35F00E0E58EC35F012006C0E58EC06
:109CA00035F0920E58EC35F0920E58EC35F0920EDD
:109CB00058EC35F06C0E58EC35F012004C0E58ECA8
:109CC00035F0920E58EC35F0920E58EC35F0920EBD
:109CD00058EC35F07C0E58EC35F012003C0E58EC88
:109CE00035F0420E58EC35F0420E58EC35F0420E8D
:109CF00058EC35F03C0E58EC35F01200000E58ECE4
:109D000035F0440E58EC35F07E0E58EC35F0400E30
:109D100058EC35F0000E58EC35F01200720E58EC8D
:109D200035F04A0E58EC35F04A0E58EC35F04A0E34
:109D300058EC35F0440E58EC35F01200220E58EC79
:109D400035F04A0E58EC35F04A0E58EC35F04A0E14
:109D500058EC35F0340E58EC35F01200300E58EC5B
:109D600035F0280E58EC35F0240E58EC35F07E0E08
:109D700058EC35F0200E58EC35F012002E0E58EC51
:109D800035F04A0E58EC35F04A0E58EC35F04A0ED4
:109D900058EC35F0320E58EC35F012003C0E58EC11
:109DA00035F04A0E58EC35F04A0E58EC35F04A0EB4
:109DB00058EC35F0300E58EC35F01200060E58EC29
:109DC00035F0020E58EC35F0620E58EC35F0120EFC
:109DD00058EC35F00E0E58EC35F01200340E58ECFD
:109DE00035F04A0E58EC35F04A0E58EC35F04A0E74
:109DF00058EC35F0340E58EC35F012000C0E58ECDF
:109E000035F0520E58EC35F0520E58EC35F0520E3B
:109E100058EC35F03C0E58EC35F01200C30E58ECFF
:109E200035F0BD0E58EC35F0BD0E58EC35F0BD0EDA
:109E300058EC35F0C30E58EC35F01200FF0E58EC1C
:109E400035F0BB0E58EC35F0810E58EC35F0BF0EF6
:109E500058EC35F0FF0E58EC35F012008D0E58EC32
:109E600035F0B50E58EC35F0B50E58EC35F0B50EB2
:109E700058EC35F0BB0E58EC35F01200DD0E58EC06
:109E800035F0B50E58EC35F0B50E58EC35F0B50E92
:109E900058EC35F0CB0E58EC35F01200CF0E58ECE4
:109EA00035F0D70E58EC35F0DB0E58EC35F0810E5E
:109EB00058EC35F0DF0E58EC35F01200D10E58ECAE
:109EC00035F0B50E58EC35F0B50E58EC35F0B50E52
:109ED00058EC35F0CD0E58EC35F01200C30E58ECAE
:109EE00035F0B50E58EC35F0B50E58EC35F0B50E32
:109EF00058EC35F0CF0E58EC35F01200F90E58EC56
:109F000035F0FD0E58EC35F09D0E58EC35F0ED0EA9
:109F100058EC35F0F10E58EC35F01200CB0E58EC41
:109F200035F0B50E58EC35F0B50E58EC35F0B50EF1
:109F300058EC35F0CB0E58EC35F01200F30E58EC1F
:109F400035F0AD0E58EC35F0AD0E58EC35F0AD0EE9
:109F500058EC35F0C30E58EC35F01200F80E58EC02
:109F600035F0240E58EC35F0220E58EC35F0240E66
:109F700058EC35F0F80E58EC35F01200FE0E58ECA7
:109F800035F0920E58EC35F0920E58EC35F0920EFA
:109F900058EC35F06C0E58EC35F012007C0E58EC95
:109FA00035F0820E58EC35F0820E58EC35F0820E0A
:109FB00058EC35F0440E58EC35F01200FE0E58EC1B
:109FC00035F0820E58EC35F0820E58EC35F0820EEA
:109FD00058EC35F07C0E58EC35F01200FE0E58ECC3
:109FE00035F0920E58EC35F0920E58EC35F0920E9A
:109FF00058EC35F0820E58EC35F01200FE0E58EC9D
:10A0000035F0120E58EC35F0120E58EC35F0120EF9
:10A0100058EC35F0020E58EC35F012007C0E58EC7E
:10A0200035F0820E58EC35F0820E58EC35F0920E79
:10A0300058EC35F0740E58EC35F01200FE0E58EC6A
:10A0400035F0100E58EC35F0100E58EC35F0100EBF
:10A0500058EC35F0FE0E58EC35F01200000E58ECBE
:10A0600035F0820E58EC35F0FE0E58EC35F0820ECD
:10A0700058EC35F0000E58EC35F01200600E58EC3C
:10A0800035F0800E58EC35F0800E58EC35F0800E2F
:10A0900058EC35F07E0E58EC35F01200FE0E58EC00
:10A0A00035F0100E58EC35F0280E58EC35F0440E13
:10A0B00058EC35F0820E58EC35F01200FE0E58ECDC
:10A0C00035F0800E58EC35F0800E58EC35F0800EEF
:10A0D00058EC35F0800E58EC35F01200FE0E58ECBE
:10A0E00035F0040E58EC35F0080E58EC35F0040E3F
:10A0F00058EC35F0FE0E58EC35F01200FE0E58EC20
:10A1000035F0080E58EC35F0100E58EC35F0200EF6
:10A1100058EC35F0FE0E58EC35F012007C0E58EC81
:10A1200035F0820E58EC35F0820E58EC35F0820E88
:10A1300058EC35F07C0E58EC35F01200FE0E58EC61
:10A1400035F0120E58EC35F0120E58EC35F0120EB8
:10A1500058EC35F00C0E58EC35F012007C0E58EC33
:10A1600035F0820E58EC35F0A20E58EC35F0420E68
:10A1700058EC35F0BC0E58EC35F01200FE0E58ECE1
:10A1800035F0120E58EC35F0120E58EC35F0120E78
:10A1900058EC35F0EC0E58EC35F012004C0E58EC43
:10A1A00035F0920E58EC35F0920E58EC35F0920ED8
:10A1B00058EC35F0640E58EC35F01200020E58ECF5
:10A1C00035F0020E58EC35F0FE0E58EC35F0020E6C
:10A1D00058EC35F0020E58EC35F012007E0E58ECBB
:10A1E00035F0800E58EC35F0800E58EC35F0800ECE
:10A1F00058EC35F07E0E58EC35F012000E0E58EC8F
:10A2000035F0300E58EC35F0C00E58EC35F0300E0D
:10A2100058EC35F00E0E58EC35F012001E0E58ECCE
:10A2200035F0E00E58EC35F0180E58EC35F0E00E35
:10A2300058EC35F01E0E58EC35F01200C60E58ECF6
:10A2400035F0280E58EC35F0100E58EC35F0280E8D
:10A2500058EC35F0C60E58EC35F012000E0E58ECE6
:10A2600035F0100E58EC35F0E00E58EC35F0100ECD
:10A2700058EC35F00E0E58EC35F01200C20E58ECCA
:10A2800035F0A20E58EC35F0920E58EC35F08A0EEF
:10A2900058EC35F0860E58EC35F01200780E58EC7C
:10A2A00035F0140E58EC35F0120E58EC35F0140E53
:10A2B00058EC35F0780E58EC35F012007E0E58EC64
:10A2C00035F04A0E58EC35F04A0E58EC35F04A0E8F
:10A2D00058EC35F0340E58EC35F012003C0E58ECCA
:10A2E00035F0420E58EC35F0420E58EC35F0420E87
:10A2F00058EC35F0240E58EC35F012007E0E58EC78
:10A3000035F0420E58EC35F0420E58EC35F0420E66
:10A3100058EC35F03C0E58EC35F012007E0E58EC3F
:10A3200035F04A0E58EC35F04A0E58EC35F04A0E2E
:10A3300058EC35F0420E58EC35F012007E0E58EC19
:10A3400035F00A0E58EC35F00A0E58EC35F00A0ECE
:10A3500058EC35F0020E58EC35F012003C0E58EC7B
:10A3600035F0420E58EC35F0420E58EC35F0520EF6
:10A3700058EC35F0340E58EC35F012007E0E58ECE7
:10A3800035F0080E58EC35F0080E58EC35F0080E94
:10A3900058EC35F07E0E58EC35F01200000E58ECFB
:10A3A00035F0420E58EC35F07E0E58EC35F0420E8A
:10A3B00058EC35F0000E58EC35F01200300E58EC29
:10A3C00035F0400E58EC35F0400E58EC35F0400EAC
:10A3D00058EC35F03E0E58EC35F012007E0E58EC7D
:10A3E00035F0100E58EC35F0080E58EC35F0140E20
:10A3F00058EC35F0620E58EC35F012007E0E58EC39
:10A4000035F0400E58EC35F0400E58EC35F0400E6B
:10A4100058EC35F0400E58EC35F012007E0E58EC3A
:10A4200035F0040E58EC35F0080E58EC35F0040EFB
:10A4300058EC35F07E0E58EC35F012007E0E58ECDC
:10A4400035F0040E58EC35F0180E58EC35F0200EAF
:10A4500058EC35F07E0E58EC35F012003C0E58ECFE
:10A4600035F0420E58EC35F0420E58EC35F0420E05
:10A4700058EC35F03C0E58EC35F012007E0E58ECDE
:10A4800035F0120E58EC35F0120E58EC35F0120E75
:10A4900058EC35F00C0E58EC35F012003C0E58EC30
:10A4A00035F0420E58EC35F0520E58EC35F0220ED5
:10A4B00058EC35F05C0E58EC35F012007E0E58EC7E
:10A4C00035F0120E58EC35F0120E58EC35F0120E35
:10A4D00058EC35F06C0E58EC35F01200440E58EC88
:10A4E00035F04A0E58EC35F04A0E58EC35F04A0E6D
:10A4F00058EC35F0320E58EC35F01200020E58ECE4
:10A5000035F0020E58EC35F07E0E58EC35F0020EA8
:10A5100058EC35F0020E58EC35F012003E0E58ECB7
:10A5200035F0400E58EC35F0400E58EC35F0400E4A
:10A5300058EC35F03E0E58EC35F01200060E58EC93
:10A5400035F0180E58EC35F0600E58EC35F0180E5A
:10A5500058EC35F0060E58EC35F012007E0E58EC33
:10A5600035F0200E58EC35F0100E58EC35F0200E7A
:10A5700058EC35F07E0E58EC35F01200460E58ECD3
:10A5800035F0280E58EC35F0100E58EC35F0280E4A
:10A5900058EC35F0460E58EC35F01200060E58EC2B
:10A5A00035F0080E58EC35F0700E58EC35F0080E0A
:10A5B00058EC35F0060E58EC35F01200440E58EC0D
:10A5C00035F0640E58EC35F0540E58EC35F04C0E66
:10A5D00058EC35F0440E58EC35F01200870E58EC6C
:10A5E00035F0EB0E58EC35F0ED0E58EC35F0EB0E87
:10A5F00058EC35F0870E58EC35F01200810E58EC0F
:10A6000035F0B50E58EC35F0B50E58EC35F0B50E0A
:10A6100058EC35F0CB0E58EC35F01200C30E58EC68
:10A6200035F0BD0E58EC35F0BD0E58EC35F0BD0ED2
:10A6300058EC35F0DB0E58EC35F01200810E58EC7A
:10A6400035F0BD0E58EC35F0BD0E58EC35F0BD0EB2
:10A6500058EC35F0C30E58EC35F01200810E58EC72
:10A6600035F0B50E58EC35F0B50E58EC35F0B50EAA
:10A6700058EC35F0BD0E58EC35F01200810E58EC58
:10A6800035F0F50E58EC35F0F50E58EC35F0F50ECA
:10A6900058EC35F0FD0E58EC35F01200C30E58ECB6
:10A6A00035F0BD0E58EC35F0BD0E58EC35F0AD0E62
:10A6B00058EC35F0CB0E58EC35F01200810E58EC0A
:10A6C00035F0F70E58EC35F0F70E58EC35F0F70E84
:10A6D00058EC35F0810E58EC35F01200FF0E58ECB6
:10A6E00035F0BD0E58EC35F0810E58EC35F0BD0E4E
:10A6F00058EC35F0FF0E58EC35F01200CF0E58EC48
:10A7000035F0BF0E58EC35F0BF0E58EC35F0BF0EEB
:10A7100058EC35F0C10E58EC35F01200810E58ECB3
:10A7200035F0EF0E58EC35F0F70E58EC35F0EB0E37
:10A7300058EC35F09D0E58EC35F01200810E58ECB7
:10A7400035F0BF0E58EC35F0BF0E58EC35F0BF0EAB
:10A7500058EC35F0BF0E58EC35F01200810E58EC75
:10A7600035F0FB0E58EC35F0F70E58EC35F0FB0EDB
:10A7700058EC35F0810E58EC35F01200810E58EC93
:10A7800035F0FB0E58EC35F0E70E58EC35F0DF0EE7
:10A7900058EC35F0810E58EC35F01200C30E58EC31
:10A7A00035F0BD0E58EC35F0BD0E58EC35F0BD0E51
:10A7B00058EC35F0C30E58EC35F01200810E58EC11
:10A7C00035F0ED0E58EC35F0ED0E58EC35F0ED0EA1
:10A7D00058EC35F0F30E58EC35F01200C30E58EC7F
:10A7E00035F0BD0E58EC35F0AD0E58EC35F0DD0E01
:10A7F00058EC35F0A30E58EC35F01200810E58ECF1
:10A8000035F0ED0E58EC35F0ED0E58EC35F0ED0E60
:10A8100058EC35F0930E58EC35F01200BB0E58ECA6
:10A8200035F0B50E58EC35F0B50E58EC35F0B50EE8
:10A8300058EC35F0CD0E58EC35F01200FD0E58EC0A
:10A8400035F0FD0E58EC35F0810E58EC35F0FD0E6C
:10A8500058EC35F0FD0E58EC35F01200C10E58ECF6
:10A8600035F0BF0E58EC35F0BF0E58EC35F0BF0E8A
:10A8700058EC35F0C10E58EC35F01200F90E58ECDA
:10A8800035F0E70E58EC35F09F0E58EC35F0E70E3A
:10A8900058EC35F0F90E58EC35F01200810E58ECFA
:10A8A00035F0DF0E58EC35F0EF0E58EC35F0DF0EDA
:10A8B00058EC35F0810E58EC35F01200B90E58EC1A
:10A8C00035F0D70E58EC35F0EF0E58EC35F0D70ECA
:10A8D00058EC35F0B90E58EC35F01200F90E58EC82
:10A8E00035F0F70E58EC35F08F0E58EC35F0F70ECA
:10A8F00058EC35F0F90E58EC35F01200000E58EC1B
:10A9000035F0000E58EC35F0040E58EC35F00A0E18
:10A9100058EC35F0040E58EC35F01200000E58ECEF
:10A9200035F0000E58EC35F0000E58EC35F0000E06
:10A9300058EC35F0000E58EC35F01200FF0E58ECD4
:10A9400035F0FF0E58EC35F0FF0E58EC35F0FF0EE9
:10A9500058EC35F0FF0E58EC35F01200280E58EC8C
:10A9600035F01200280E58EC35F0280E58EC35F072
:10A97000280E58EC35F0280E58EC35F0280E58EC1F
:10A9800035F01200100E58EC35F0100E58EC35F082
:10A990007C0E58EC35F0100E58EC35F0100E58ECDB
:10A9A00035F01200100E58EC35F0100E58EC35F062
:10A9B000100E58EC35F0100E58EC35F0100E58EC27
:10A9C00035F01200EF0E58EC35F0EF0E58EC35F084
:10A9D000EF0E58EC35F0EF0E58EC35F0EF0E58EC6A
:10A9E00035F01200400E58EC35F0200E58EC35F0E2
:10A9F000100E58EC35F0080E58EC35F0040E58ECFB
:10AA000035F01200BF0E58EC35F0DF0E58EC35F083
:10AA1000EF0E58EC35F0F70E58EC35F0FB0E58EC15
:10AA200035F01200FE0E58EC35F0FE0E58EC35F005
:10AA3000000E58EC35F01200000E58EC35F0000E08
:10AA400058EC35F0000E58EC35F01200000EAA6EEE
:10AA5000000EA96E1150A86EA69EA69CA684550E47
:10AA6000A76EAA0EA76EA682A6B234EF55F0A694E2
:10AA70001200000EAA6E010EA96E1250A86EA69EBC
:10AA8000A69CA684550EA76EAA0EA76EA682A6B295
:10AA900047EF55F0A6941200000EAA6E020EA96EA2
:10AAA0001350A86EA69EA69CA684550EA76EAA0E4D
:10AAB000A76EA682A6B25AEF55F0A6941200000E19
:10AAC000AA6E030EA96E1450A86EA69EA69CA6841C
:10AAD000550EA76EAA0EA76EA682A6B26DEF55F010
:10AAE000A6941200000EAA6E040EA96E1550A86E50
:10AAF000A69EA69CA684550EA76EAA0EA76EA68239
:10AB0000A6B280EF55F0A6941200000EAA6E050EB4
:10AB1000A96E1650A86EA69EA69CA684550EA76E7A
:10AB2000AA0EA76EA682A6B293EF55F0A6941200C5
:10AB3000000EAA6E060EA96E1750A86EA69EA69CC1
:10AB4000A684550EA76EAA0EA76EA682A6B2A6EF81
:10AB500055F0A6941200000EAA6E070EA96E1850AA
:10AB6000A86EA69EA69CA684550EA76EAA0EA76EDA
:10AB7000A682A6B2B9EF55F0A6941200000EAA6EF6
:10AB8000080EA96E1950A86EA69EA69CA684550E06
:10AB9000A76EAA0EA76EA682A6B2CCEF55F0A69419
:10ABA0001200000EAA6E090EA96E1A50A86EA69E7B
:10ABB000A69CA684550EA76EAA0EA76EA682A6B264
:10ABC000DFEF55F0A6941200000EAA6E0A0EA96ED1
:10ABD0004D9E4D50A86EA69EA69CA684550EA76EAF
:10ABE000AA0EA76EA682A6B2F3EF55F0A6941200A5
:10ABF000000EAA6E0B0EA96E5F50A86EA69EA69CB4
:10AC0000A684550EA76EAA0EA76EA682A6B206EF60
:06AC100056F0A6941200AC
:020000040030CA
:03000100331800B1
:02000500358044
:060008000FC00FE00F40E5
:0200000400F00A
:0C00000008044BBB9B887F7F00000000C1
:00000001FF
